:100000000C941E060C9431280C945E280C94460621
:100010000C9446060C9446060C9446060C94460630
:100020000C9446060C9446060C94EF120C9446066B
:100030000C9446060C9446060C9446060C94460610
:100040000C948B280C9446060C94792C0C94BC2CA4
:100050000C9446060C9446060C9446060C944606F0
:100060000C9446060C9446069F180119E018E318F4
:10007000E618E918EC18EF18F2180119FB18331AF2
:10008000351A351A331A351A351A351A351A351AFA
:10009000351A351A351A351A351A351A351A351AE8
:1000A000B919351A351A351A351A351A2A19351A61
:1000B000351A351A351A351A351A351A351A351AC8
:1000C000351A351A351A351A351A351AC519C5199A
:1000D000C519C519C519C519C519C519C519351ABF
:1000E000351A351A351A351A351A2A19C419C41988
:1000F000C419C419351AD219D819DE19E419EA1924
:10010000F019F619FC19061A101A1A1A241A6B1982
:100110002D19351A351A351A351AB919351A351AED
:10012000351A351A351A351A351A351AC319C3193D
:10013000C319C319351AD219D819DE19E419EA19E5
:10014000F019F619FC19061A101A1A1A241A6B1942
:100150002D19351A351A351A351AB919681A681A47
:10016000681A681A681A681A681A681A681A681A7F
:10017000681A681A681A7F1B7F1B7F1B7F1B7F1BF7
:100180007F1BAD1AB71AC11ACB1A291B331B421B8E
:10019000531BDB1CF01CFC1C051D141D391D421DCE
:1001A0008B1D541D9F20A520AB20B220C020E22033
:1001B0000021456E746572206D656E752E2E2E00C1
:1001C000546F67676C6564206D6963726F50504D42
:1001D00000546F67676C656420696E76657274653C
:1001E000642050504D2100546F67676C6564205443
:1001F00058206D7574696E672100546F67676C6570
:10020000642074656C656D65747279210050726F3D
:10021000746F636F6C206572726F72207769746897
:100220002052580054696D656F7574207768656E4B
:1002300020636F6E6E656374696E6720746F205201
:100240005800507265737320616E79206B65792058
:10025000746F2063616E63656C00436F6E6E6563DF
:1002600074696E6720746F2052582C20706F776508
:100270007220757020746865205258202877697440
:10028000682062696E6420706C7567206966206EF4
:100290006F74207573696E6720616C776179732064
:1002A00062696E642900546F67676C656420276912
:1002B0006D6D656469617465206F75747075742700
:1002C00000546F67676C65642027736C61766520E6
:1002D0006D6F64652700546F67676C6564202761E4
:1002E0006C776179732062696E642700546F676769
:1002F0006C65642050504D206368616E6E656C20A3
:100300006C696D69740053657420525353492069B8
:100310006E6A656374696F6E206368616E6E656C8A
:100320002028303D3D64697361626C652900536526
:10033000742050504D206D696E696D756D20737914
:100340006E630053657420626561636F6E20696E31
:1003500074657276616C0053657420626561636FC9
:100360006E2064656C617900536574206265616319
:100370006F6E206672657175656E637920696E2097
:10038000487A3A20303D64697361626C652C205074
:10039000783D504D52206368616E6E656C20782CFC
:1003A0002046783D465253206368616E6E656C202E
:1003B00078005365742050574D2073746F7020641B
:1003C000656C61792028302064697361626C6564B2
:1003D0002C20312D323535203D3D20302E317320FB
:1003E0002D2035306D696E29005365742050504DB5
:1003F0002073746F702064656C61792028302064EC
:10040000697361626C65642C20312D323535203D75
:100410003D20302E3173202D2035306D696E29003E
:10042000536574206661696C736166652064656CF0
:1004300061792028302064697361626C65642C20C6
:10044000312D323535203D3D20302E3173202D2089
:1004500035306D696E29002A2A2A2A2A2A2A2A2A50
:100460002A2A2A2A2A2A2A2A2A2A2A2A2A2A2A2AEC
:100470002A2A2A2A0052582041636B6564202D20C5
:1004800072657665727420737563636573736675E0
:100490006C21002A2A2A2A2A2A2A2A2A2A2A2A2AAD
:1004A0002A2A2A2A2A2A2A2A2A2A2A2A2A2A2A2AAC
:1004B000002A2A2A2A2A2A2A2A2A2A2A2A2A2A2AC6
:1004C0002A2A2A2A2A2A2A2A2A2A2A2A2A2A00528E
:1004D000582041636B6564202D20757064617465DC
:1004E000207375636365737366756C21002A2A2A0D
:1004F0002A2A2A2A2A2A2A2A2A2A2A2A2A2A2A2A5C
:100500002A2A2A2A2A2A2A2A2A2A0056616C696457
:100510002063686F69636573206172653A205B319F
:100520005D2D5B31365D20286368616E6E656C20E1
:10053000312D31362900536574206F7574707574D0
:1005400020666F7220706F727420005B585D2061AE
:10055000626F7274206368616E67657320616E6498
:10056000206578697420525820636F6E6669670051
:100570005B535D20736176652073657474696E6783
:100580007320746F205258005B525D20726576654F
:1005900072742052582073657474696E6773207486
:1005A0006F2064656661756C747300557365206EA9
:1005B000756D62657273205B312D445D20746F2010
:1005C0006564697420706F727473205B452D515D92
:1005D00020666F722073657474696E677300202DD6
:1005E00020726563656976657220636F6E66696700
:1005F000757261746F722C20727820737720000AF4
:100600000A6F70656E4C52536E67200053657420FC
:1006100073657269616C2062617564726174653AB8
:10062000200056616C69642063686F696365733A82
:100630002031202D20342B34202F2032202D203823
:10064000202F2033202D20382B34202F2034202D14
:10065000203132202F2035202D2031322B34202FF5
:100660002036202D20313600536574204368616E9A
:100670006E656C20636F6E6669673A20005365741F
:100680002044617461726174652028302D32293AEA
:10069000200053657420486F70206368616E6E653A
:1006A0006C7320286D61782032342C207365706162
:1006B000726174656420627920636F6D6D61732966
:1006C0002076616C69642076616C75657320312DCC
:1006D0003235353A2000536574206368616E6E656B
:1006E0006C2073706163696E6720287831306B48C5
:1006F0007A293A200053657420524620706F77653E
:10070000722028302D37293A200053657420524634
:10071000206D6167696320286865782920652E67E8
:100720002E20307844454144463030443A2000532E
:1007300065742062617365206672657175656E63AC
:10074000792028696E20487A293A20005B5A5D207A
:10075000656E746572207265636569766572206383
:100760006F6E66696775726174696F6E2075746902
:100770006C79005B465D20646973706C61792061FF
:10078000637475616C206672657175656E63696509
:10079000732075736564005B525D2063616C6375E3
:1007A0006C6174652072616E646F6D206B65792079
:1007B000616E6420686F70206C697374005B495DC2
:1007C000207265696E697469616C697A6520736508
:1007D0007474696E677320746F20736B65746368DB
:1007E0002064656661756C7473005B585D2072658A
:1007F00076657274206368616E67657320616E64EC
:100800002065786974206D656E75005B535D20739B
:100810006176652073657474696E677320746F20E8
:10082000454550524F4D20616E64206578697420B3
:100830006D656E7500557365206E756D62657273BA
:10084000205B302D395D20746F20656469742070E1
:100850006172616D657465727300202D2053797328
:1008600074656D20636F6E66696775726174696F18
:100870006E000A0A6F70656E4C52536E672000510D
:1008800029204F7574707574206265666F726520DB
:100890006C696E6B20283D465329203A2000502970
:1008A00020536C617665206D6F64652028657870D3
:1008B0006572696D656E74616C293A20004F29205C
:1008C00054696D65642042494E44206174207374FC
:1008D000617274757020203A20004E292050504DCE
:1008E000206F7574707574206C696D69746564200F
:1008F000202020203A200044495341424C454400E6
:100900004D292050504D205253534920746F20637D
:1009100068616E6E656C202020203A20004C2920F2
:1009200050504D206D696E696D756D2073796E63E1
:10093000202875732920203A200044495341424C15
:100940004544004B29204661696C736166652062ED
:100950006561636F6E20696E74762E2028312D32AA
:10096000353573293A20004A29204661696C736144
:10097000666520626561636F6E2064656C617920D5
:1009800028302D323535203D3E20313073202D204A
:100990003135306D696E293A200049292046616958
:1009A0006C7361666520626561636F6E206672714B
:1009B0002E203A200048292050574D2073746F7024
:1009C0002064656C6179202020202020203A2000BE
:1009D00047292050504D2073746F702064656C61FE
:1009E00079202020202020203A200046292046611E
:1009F000696C736166652064656C617920202020D4
:100A00002020203A200050574D206368616E6E65AB
:100A10006C200066756E6374696F6E3A2000292041
:100A2000706F72742000506F776572546F776572C3
:100A300000445446205548462033322D62697420C4
:100A400031306368004F70656E4C52536E67525878
:100A5000206D696E6920342F36636800466C7974A6
:100A6000726F6E2F4F72616E6765525820554846FF
:100A70002038636800525820747970653A20004429
:100A8000697361626C656400487A00203D3D200016
:100A900043616C63756C61746564207061636B6540
:100AA0007420696E74657276616C3A200042292068
:100AB0004D6963726F202868616C66292050504D23
:100AC000202020203A00412920496E766572746505
:100AD000642050504D20696E20202020203A0030A4
:100AE00029204D7574652062757A7A657220286DAB
:100AF0006F73746C79293A003929205365726961E2
:100B00006C2062617564726174653A00736D617224
:100B100074506F7274004672536B79005472616E38
:100B200073706172656E740044697361626C6564B0
:100B30000038292054656C656D657472793A2020FF
:100B40002020202020003729204368616E6E656CCC
:100B500020636F6E6669673A202000362920446161
:100B60007461726174652028302D32293A2020206A
:100B700000352920486F70206368616E6E656C7364
:100B80003A2020202020003429204368616E6E65C1
:100B90006C2073706163696E673A202000332920EE
:100BA000524620706F7765722028302D37293A2001
:100BB0002020003229205246206D616769633A2067
:100BC0002020202020202020003129204261736530
:100BD000206672657175656E63793A202020000089
:100BE00000000700020100000304060000000000EE
:100BF00000000001020408102040800102040810D7
:100C00002001020408102004040404040404040263
:100C10000202020202030303030303000000002395
:100C2000002600290000000000250028002B0000FD
:100C3000000000240027002A0000302E11241FBECF
:100C4000CFEFD8E0DEBFCDBF13E0A0E0B1E0EEE62D
:100C5000F2E602C005900D92A83CB107D9F716E064
:100C6000A8ECB3E001C01D92A239B107E1F71CE086
:100C7000CCE3DCE004C02297FE010E94392FCA3386
:100C8000D107C9F70E946C2E0C9435310C940000EA
:100C900080917705813019F482E080937705809107
:100CA0007705833019F484E0809377050895A8953B
:100CB0000895DC01ED91FC910190F081E02D099502
:100CC00008952091780530917905382748E0C901C9
:100CD000880F991F37FF06C09C0151E2252750E17C
:100CE000352701C09C01415091F73093790520933D
:100CF0007805089588E380937A0580E092ECA1E07E
:100D0000B0E080937B0590937C05A0937D05B09324
:100D10007E0587E08093870580EC92E9ADEEB9E12E
:100D200080937F0590938005A0938105B093820501
:100D300085E0809388058DEE9EEFADEABEED809351
:100D4000830590938405A0938505B0938605E9E813
:100D5000F5E080E090E0863028F4DC01AE54BC4F32
:100D60002C9101C020E0219301968831910599F7DB
:100D700082E08093A1058AE08093A205089580EC2B
:100D800091EDA8E9BBE18093BF059093C005A093C6
:100D9000C105B093C20580E090E0A0E0B0E580938B
:100DA000C3059093C405A093C505B093C605E7ECB1
:100DB000F5E080E081938F5F8031E1F70895A0E056
:100DC000B0E0E5EEF6E00C94022FD82F0E94E12867
:100DD0006115710581059105C9F30E94A52F109237
:100DE0008305109284051092850510928605C4E053
:100DF000812C912C54018A94C0908305D090840555
:100E0000E0908505F0908605FE2CED2CDC2CCC24A2
:100E10000E94A02FA50194010E94E12E6C0D7D1D62
:100E20008E1D9F1D609383057093840580938505B7
:100E300090938605C15001F7DD2309F450C009E8FD
:100E400015E0E801A12CB12C62E3C62ED12CE12CD7
:100E5000F12C8881882309F442C0B39419F40E94CC
:100E60007A063DC00E94A02FA70196010E94E12EA4
:100E7000E1E0E60FA9E8B5E08A2F801B8A1520F48F
:100E80008D918E13F9CFE9CF2091880530E0A0E154
:100E9000B7E20E94792E9B01AC01AE2FB0E00E9418
:100EA000882E40907F05509080056090810570905D
:100EB0008205640D751D861D971D4090BF055090DD
:100EC000C0056090C1057090C205461657066806B9
:100ED000790618F2E993A39488E1A812BACFCDB7A6
:100EE000DEB7E0E10C941E2F8436910520F4BC019E
:100EF00080E090E017C09C018E3B910528F42A55B4
:100F00003109AAE0B0E00CC0823D910528F4245BD1
:100F10003109A4E6B0E004C02D5C3109A8E5B2E0D7
:100F20000E94792EA4E6B0E09B01AC010E94882EBD
:100F3000089590E08C599F4F0E947407089561E0D6
:100F40008AE00E948E2960E08AE00E94C729089505
:100F5000892B11F061E001C060E08AE00E94C7299E
:100F6000089560E08CE00E948E2961E08BE00E9491
:100F70008E2961E08DE00E948E2960E082E00E946F
:100F80008E2961E084E00E948E29089542E050E0BD
:100F900068E476E080E00E9411280895E3E0F0E044
:100FA00089E080935700E491E67081E0E63009F033
:100FB00080E00895CF93DF93C82F0E94CE07882347
:100FC00081F0DFB781E080937605F8940E945706A0
:100FD00088E180936000C0936000C1110E945706B1
:100FE000DFBFDF91CF9108958F929F92AF92BF9212
:100FF000CF92DF92EF92FF92CF93FC01C0A5EC2F2E
:10100000E770F0E0E658FC4FA081B0E0C7FF03C0F6
:1010100024E130E002C02FE030E0FC0197A183E141
:10102000989FF0011124E25CFE4F80809180A280A5
:10103000B380A20FB31F20E43FE14DE750E00E94D0
:10104000932EA50194010E94BF2E8C2F887149F424
:1010500069017A01E0EDCE0EE7E0DE1EE11CF11C35
:101060001BC0C7FF05C060E47AE88CE29EE004C0C4
:1010700060E07EEE8AEB9BE069017A01F8EBCF0E2F
:10108000FBE0DF1EE11CF11CA50194010E94BF2EB4
:10109000C20ED31EE41EF51EC701B60169517C4F76
:1010A0008F4F9F4F28EE33E040E050E00E94BF2E6C
:1010B000A8EEB3E00E94882ECF91FF90EF90DF90D2
:1010C000CF90BF90AF909F908F9008958F3F9105E4
:1010D00051F048F0811522E0920738F081159340D5
:1010E00030F482E0089580E0089581E0089583E07F
:1010F0000895A0E0B0E0EFE7F8E00C940B2FEB01CF
:101100008A01B82FB695A0E028813981F8012083A3
:101110002A813B8121832C813D8122832E813F8145
:101120002383688179814A815B812C813D81EE81B5
:10113000FF819F2F9295990F990F907C272F2370F5
:10114000922B252F2370220F220F922B232F2370F7
:101150002295207F922BF80194830B5F1F4F2896D6
:10116000AF5FBA1788F680FF24C0888199810E94FA
:101170006608D82E8A819B810E946608E82E8C81A1
:101180009D810E946608F82E8E819F810E946608CC
:10119000F0E4DF9EA001112490E1E99E900111246A
:1011A000242B282BE4E0FE9EB0011124262BF8010D
:1011B0002083CDB7DEB7E7E00C94272F803223E001
:1011C000920708F1883E23E0920740F48F51934044
:1011D000E4E096958795EA95E1F70895803D27E04C
:1011E000920718F48C5D93400895883928E092079F
:1011F00068F4885C974074E0969587957A95E1F756
:101200008D509C4F089580E090E008958FEF93E01B
:1012100008958C30910540F4A4E0880F991FAA9599
:10122000E1F7885D9C4F0895843F23E0920718F40E
:1012300084529C4F0895811524E0920740F486570C
:10124000934FF4E0880F991FFA95E1F7089580E92C
:1012500098E008959C013695279525753575821B74
:10126000930B9C0123733373969587959695879579
:1012700083739373820F931F9C0154E036952795D7
:101280005A95E1F7280F391F2F703F7041E051E068
:10129000249FC001259F900D349F900D1124892F0C
:1012A00008952D98882319F000002B9A02C00000A1
:1012B0002B9800002D9A000008952D9A000083B10C
:1012C0002D980000829581700895CF93DF93D82FD9
:1012D0005C9A2D985C98C8E08D2F80780E94510907
:1012E000DD0FC150C9F72D98DF91CF9108958F7709
:1012F0000E9465090895CF93DF93D82FC8E08D2F02
:1013000080780E945109DD0FC150C9F72D98DF91F7
:10131000CF910895CF93DF932D98C8E080E0D82F28
:10132000DD0F0E945D098D0FC150C9F7DF91CF918C
:1013300008950E9477090E948A095C9A0895A1E0A5
:10134000B0E0E5EAF9E00C94102F806869830E9410
:1013500065096981862F0E947B095C9A2196E2E0EB
:101360000C942C2FCF93C0918305C827E82FF0E071
:10137000E658FA4F678589E70E949F096C2F8DE335
:101380000E949F096C2F82E40E949F09CF910895CB
:1013900086E20E9499090895CF93DF93EC016C8156
:1013A0008CE10E949F096D818DE10E949F096E81F1
:1013B0008EE10E949F096F8180E20E949F096885EB
:1013C00081E20E949F09698582E20E949F096A85E5
:1013D00083E20E949F096B8584E20E949F096C85CD
:1013E00085E20E949F096D858AE20E949F096E85B1
:1013F0008EE60E949F096F858FE60E949F0968898B
:1014000080E70E949F09698981E70E949F096A8994
:1014100082E70E949F09DF91CF910895CF92DF92DA
:10142000EF92FF92CF93DF936B017C01C11488E3AD
:10143000D8068CE9E8068CE1F80628F5C701B60164
:1014400020E836E948E950E00E94BF2EE90168979C
:1014500060E879E687E69FEF0E949B2E6C0D7D1D6C
:101460008E1D9F1DF2E0660F771F881F991FFA954A
:10147000D1F721E732E040E050E00E94BF2EF22E8B
:10148000E32E80E421C0C701B60120E03DE241E344
:1014900051E00E94BF2EE901689760E073ED8EEC89
:1014A0009EEF0E949B2E6C0D7D1D8E1D9F1D660F55
:1014B000771F881F991F21E732E040E050E00E942B
:1014C000BF2EF22EE32E80E66C2F6F71680F85E73A
:1014D0000E949F096E2D86E70E949F096F2D87E766
:1014E0000E949F09DF91CF91FF90EF90DF90CF9006
:1014F0000895682F8DE60E949F0908958F929F920C
:10150000AF92BF92CF92DF92EF92FF92CF93DF9391
:10151000D82F83E00E9499098093750584E00E948A
:1015200099098093740560E086E00E949F0961E05C
:1015300087E00E949F096FE789E00E949F0965E0AC
:101540008AE00E949F0962E18BE00E949F0965E1A9
:101550008CE00E949F096DEF8DE00E949F0960E082
:101560008EE00E949F09DD2319F08BE291E008C014
:101570002091A10533E1239FC0011124825C9E4F7D
:101580000E94CC096CE880E30E949F096FE082E32F
:101590000E949F0962E483E30E949F098091A20553
:1015A00087FF02C064E101C06AE084E30E949F09F2
:1015B0006AE285E30E949F096DE286E30E949F092B
:1015C00064ED87E30E949F0960E088E30E949F0921
:1015D00060E089E30E949F09D11109C0C090830592
:1015E000D0908405E0908505F090860507C0C5E998
:1015F000CC2EC1ECDC2EED2CCEEDFC2ECAE38F2CD4
:101600009924AA24BB24682D8C2F0E949F09682D41
:1016100085E08C0F0E949F09FE2CED2CDC2CCC2445
:10162000CF5FCE3361F76FEF83E40E949F096FEFC6
:1016300084E40E949F096FEF85E40E949F096FEF89
:1016400086E40E949F09DD2311F066E002C06091EC
:1016500087058DE60E949F0960E089E70E949F0947
:10166000609188058AE70E949F0960E083E70E94F5
:101670009F0960E084E70E949F09D11109C0609131
:101680007F0570918005809181059091820504C04D
:1016900060EC72E98DEE99E10E940E0ADF91CF9124
:1016A000FF90EF90DF90CF90BF90AF909F908F9082
:1016B000089561E087E00E949F0964E28EE70E943E
:1016C0009F0963E088E00E949F0960E088E00E9433
:1016D0009F0965E087E00E949F0962E085E00E9423
:1016E0009F0983E00E9499098093750584E00E9418
:1016F000990980937405089583E00E949909809365
:10170000750584E00E9499098093740561E087E083
:101710000E949F096AE070E080E090E00E94042946
:101720000E94590B00000895CF92DF92FF920F9311
:101730001F93CF93DF931F92CDB7DEB7082F162FDD
:101740008EE399830E949F09F02EC02E9981D92E95
:101750008C2D8F19811738F4F60161916F018FE795
:101760000E949F09F5CF64E085E00E949F0983E015
:101770000E9499098093750584E00E9499098093DD
:1017800074050E94E1286093700570937105809341
:1017900072059093730569E087E00E949F0981E0DC
:1017A000809377050F90DF91CF911F910F91FF905C
:1017B000DF90CF9008950F931F930E94940B809118
:1017C0007705813099F40E94E1280091700510910D
:1017D00071052091720530917305601B710B820BAE
:1017E000930B603A76488140910548F380917705E4
:1017F000813031F46EE971E086EE95E00E94CD2AE9
:101800001F910F9108950F931F9380917705823058
:1018100021F41092770581E020C080917705813016
:10182000D9F40E94E1280091700510917105209172
:10183000720530917305601B710B820B930B613A3B
:1018400076488140910540F061E087E00E949F0961
:101850001092770582E001C080E01F910F910895FA
:10186000CF93DF93EC014AE050E06D2F70E086EEFD
:1018700095E00E949B2B6EE286EE95E00E949F2AE7
:10188000BE0184E0769567958A95E1F76F707727BA
:101890004AE050E086EE95E00E949B2B6EE286EED9
:1018A00095E00E949F2ABE016F7077274AE050E0C2
:1018B00086EE95E00E949B2BDF91CF910895D82F63
:1018C000C0E0CD1790F45E9A409A64E670E080E044
:1018D00090E00E9404295E98409864E670E080E001
:1018E00090E00E940429CF5FECCF6CE271E080E0D1
:1018F00090E00E940429E4CF0F931F93CF93DF93CE
:10190000EC01062F15E0115051F0CE010E941C3160
:10191000081741F0602FCE010E942431F4CF82E0FD
:101920000E945F0CDF91CF911F910F910895A0E06D
:10193000B0E0EDE9FCE00C94022F482E562EC0E0FA
:10194000D0E0612C712CE12CF12C00E010E0411072
:101950000CC06090D80586E4689E3001112459E1DE
:10196000E52EF12C0EEB15E01EC091E049120FC0E0
:101970006090D805E6E46E9E30011124FBE16F0E05
:10198000711C49E2E42EF12C0AE715E00CC082E05C
:10199000481209C028E1622E77247394EE24E39460
:1019A000F12C07ED15E043018C0E9D1E1092790578
:1019B000109278053401A62CA818B12CC301019609
:1019C0006C01AE14BF04A8F4A00EB11E511006C0E5
:1019D000C3010E941C31F501808305C0F5016081BF
:1019E000C3010E947C0CF50180810E9461063601D2
:1019F000E2CFC301511018C0C3010E941C31B82EA0
:101A0000C6010E941C312B2D30E0322F2227282BBB
:101A100080917805909179058217930779F4C0E059
:101A2000D0E05524539493CF3601609179050E94FC
:101A30007C0C60917805C6010E947C0CC05EDE4F74
:101A4000C13E92E0D90708F482CF852DCDB7DEB72D
:101A5000E0E10C941E2F61E082E00E94970C089553
:101A600060E082E00E94970C8091D705853020F0DD
:101A70001092D7050E942B0D8091D7058093D80531
:101A8000089561E080E00E94970C61E081E00E948F
:101A9000970C089560E080E00E94970C882351F035
:101AA00060E081E00E94970C882321F080917A0504
:101AB000883349F00E94BF060E947A0681E00E94A6
:101AC000DF060E94410D0895882319F06AEA71E04B
:101AD00002C06EEA71E086EE95E00E94CD2A08957C
:101AE000FF920F931F93CF93DF9369EC7BE086EE19
:101AF00095E00E94792A40917F0550918005609180
:101B00008105709182052AE030E086EE95E00E9422
:101B1000A22B63EB7BE086EE95E00E94792A409150
:101B2000830550918405609185057091860520E1BB
:101B300030E086EE95E00E94A22B6DE97BE086EE18
:101B400095E00E94792A4AE050E06091870586EE90
:101B500095E00E94CA2B67E87BE086EE95E00E9444
:101B6000792A4AE050E06091880586EE95E00E946F
:101B7000CA2B61E77BE086EE95E00E94792AC9E8EE
:101B8000D5E0F12C8E0188818823A9F0FF2031F067
:101B900061EB71E086EE95E00E949C2A21964AE076
:101BA00050E0F801608186EE95E00E94932BF3945B
:101BB000F8E1FF12E7CF86EE95E00E94A72A6BE5D9
:101BC0007BE086EE95E00E94792A4AE050E0609141
:101BD000A10586EE95E00E94CA2B66E47BE086EEC6
:101BE00095E00E94792AE091A205E770F0E0EE0FFF
:101BF000FF1FEE57FC4F6081718186EE95E00E94D9
:101C0000CD2A61E37BE086EE95E00E94792A8091FF
:101C1000A2058871883069F028F4811113C068E248
:101C20007BE00CC0803141F0883161F46CE07BE0F6
:101C300005C06CE17BE002C066E17BE086EE95E0EA
:101C40000E94BB2A68EF7AE086EE95E00E94792A2E
:101C500040917B0550917C0560917D0570917E05DA
:101C60002AE030E086EE95E00E94A22B6FED7AE04C
:101C700086EE95E00E94792A8091C30580710E94CA
:101C8000640D66EC7AE086EE95E00E94792A8091F8
:101C9000C30580740E94640D6DEA7AE086EE95E0DB
:101CA0000E94792A8091C30580720E94640D60E9C8
:101CB0007AE086EE95E00E94792A8AE795E00E9414
:101CC000F407AB01BC012AE030E086EE95E00E940B
:101CD000842B6BE87AE086EE95E00E94792A8AE709
:101CE00095E00E94F4079B01AC0160E472E48FE090
:101CF00090E00E94BF2EBA01A9012AE030E086EEF2
:101D000095E00E94842B68E87AE086EE95E00E94D8
:101D1000BB2ACDB7DEB7E5E00C94292F8F929F92B6
:101D2000AF92BF92CF92DF92EF92FF92811107C0E4
:101D30006FE77AE086EE95E00E94BB2A2FC090E024
:101D40000E94740724E630E040E050E00E94BF2E7D
:101D5000CA01B9012AE030E040E050E00E94BF2E05
:101D600049015A016B017C012AE030E0B501A40170
:101D700086EE95E00E94842B6EE286EE95E00E944E
:101D80009F2A2AE030E0B701A60186EE95E00E9486
:101D9000842B63E786EE95E00E94DF2AFF90EF90A8
:101DA000DF90CF90BF90AF909F908F9008951F933A
:101DB000CF93DF9365E77AE086EE95E00E94792A7B
:101DC0008091A305813041F46CE57AE086EE95E0E0
:101DD0000E94BB2A10E050C0823019F465E47AE01A
:101DE000F5CF843019F461E37AE0F0CF853091F7D4
:101DF00066E27AE0EBCFC12FD0E0C930D1050CF418
:101E000041C068E3610F86EE95E00E949F2A6EE173
:101E10007AE086EE95E00E94792ABE016F5F7F4FDF
:101E20004AE050E086EE95E00E94632B63E17AE0A1
:101E300086EE95E00E94792ACD55DA4FE981E032AD
:101E400018F566E07AE086EE95E00E94792A8981AD
:101E5000803130F06DE673E086EE95E00E949C2ABA
:101E600069816F7070E06F5F7F4F4AE050E086EEEF
:101E700095E00E946C2B1F5F80914C05181708F4A9
:101E8000BACF0FC061E3BECFEF70F0E0EE0FFF1FDF
:101E9000EE56FC4F6081718186EE95E00E94CD2A5E
:101EA000EACF6BEE79E086EE95E00E94792A809188
:101EB000BB050E948E0E60ED79E086EE95E00E94F3
:101EC000792A8091BC050E948E0E65EB79E086EE42
:101ED00095E00E94792A8091BD050E948E0E6AE9E4
:101EE00079E086EE95E00E94792A4091B305509101
:101EF000B4056091B5057091B605411551056105B0
:101F0000710539F12AE030E086EE95E00E94A22BBF
:101F100067E679E086EE95E00E94792A8091B70520
:101F20000E949907AB01BC012AE030E086EE95E003
:101F30000E94A22B63E479E086EE95E00E94792A64
:101F40004AE050E06091B80586EE95E00E94CA2B09
:101F500006C06AE379E086EE95E00E94BB2A6DE157
:101F600079E086EE95E00E94792A6091B90570913A
:101F7000BA054AE050E086EE95E00E94B42B60E09E
:101F800079E086EE95E00E94792A6091B20560348E
:101F900050F470E06F5F7F4F4AE050E086EE95E0CE
:101FA0000E946C2B06C067EF78E086EE95E00E94F9
:101FB000BB2A6AED78E086EE95E00E94792A80914E
:101FC000B10580FF03C063EB71E002C067EB71E015
:101FD00086EE95E00E94CD2A6DEB78E086EE95E0E6
:101FE0000E94792A8091B10582700E94640D6EE989
:101FF00078E086EE95E00E94792A8091B1058470A0
:102000000E94640D6FE778E086EE95E00E94792AE1
:102010008091B10588700E94640DDF91CF911F916E
:1020200008950F931F93CF93DF93209149052F3F7E
:10203000A9F56FEF75E086EE95E00E94792A88E8B1
:1020400093E00E94300C6EED75E086EE95E00E9404
:10205000792A80914A0590914B050E94300C6BEAD9
:1020600075E086EE95E00E94BB2A68E875E086EE92
:1020700095E00E94BB2A60E775E086EE95E00E943D
:10208000BB2A6BE475E086EE95E00E94BB2A86EEE3
:1020900095E00E94A72A0E94D70E68C012160CF085
:1020A00065C0332727FD309580914C0590E082175D
:1020B00093070CF45BC066E375E086EE95E00E9442
:1020C000792A60914905772767FD70954AE050E0CD
:1020D00086EE95E00E946C2B6BE075E086EE95E055
:1020E0000E94792A10E008E280914D051817D0F57A
:1020F000C12FD0E0CC0FDD1FC25BDA4F288130E06A
:1021000080914905992787FD9095019728173907F0
:1021100039F56BEB71E086EE95E00E949C2A4AE06F
:1021200050E0602F86EE95E00E94932B6FEB71E0FC
:1021300086EE95E00E949C2AE981EF70F0E0EE0FB8
:10214000FF1FEE56FC4F6081718186EE95E00E9484
:102150009C2A63EC71E086EE95E00E949C2A0F5F5A
:102160001F5FC2CF86EE95E00E94A72ADF91CF9134
:102170001F910F910895FF920F931F93CF93DF93B9
:10218000C9E8D5E0F12C8E0188818823D1F165EC76
:1021900071E086EE95E00E949C2A4AE050E06F2DA7
:1021A00086EE95E00E94932B62ED71E086EE95E05D
:1021B0000E949C2A2196F801208130E0A0E1B7E23C
:1021C0000E94792E9B01AC01A0918805B0E00E948D
:1021D000882EAB01BC0180917F0590918005A09174
:1021E0008105B0918205480F591F6A1F7B1F2AE0A5
:1021F00030E086EE95E00E94A22BF394F8E1FF1206
:10220000C2CFCDB7DEB7E5E00C94292F1092E304DE
:1022100085E6E4EEF4E0DF011D928A95E9F7089582
:10222000CF93C82F8F3719F0883009F045C0E0915F
:10223000E304EE23D9F1E150E093E304F0E0EC5144
:10224000FB4F10826DE070E086EE95E00E9459062B
:10225000C0E08091E304C81760F4EC2FF0E0EC518B
:10226000FB4F608170E086EE95E00E945906CF5FDB
:10227000F0CF60E270E086EE95E00E9459066DE0D6
:1022800070E086EE95E00E945906C0E08091E3047C
:10229000C81778F5EC2FF0E0EC51FB4F608170E04F
:1022A00086EE95E00E945906CF5FF0CF67E086EE9C
:1022B00095E00E949F2A1DC08B3119F40E940611DF
:1022C0001AC08D30C1F08A30B1F08091E3048436B9
:1022D00068F76C2F70E086EE95E00E945906E09159
:1022E000E30481E08E0F8093E304F0E0EC51FB4FB8
:1022F000C08380E001C081E0CF910895CF93C82FC3
:102300000E94E1286093CC047093CD048093CE04A6
:102310009093CF04C093E104CC2329F040E051EE28
:1023200060E070E004C040E855E260E070E086EEF6
:1023300095E00E94292DCF9108959091D004492FC6
:102340004F7050E0BA016F5F7F4F292F30E0E4E01B
:1023500035952795EA95E1F76217730759F0FA0169
:10236000EF52FB4F808381E0890F8F70907F892B24
:102370008093D00408956EE770E086EE95E00E94A9
:1023800059060895A3E1B1E0E8ECF1E10C94032FC4
:10239000E9E8F5E0712C8191882321F0739428E11C
:1023A0007212F9CF66ED71E086EE95E00E94CD2ABB
:1023B0004AE050E0672D86EE95E00E94CA2B80E04F
:1023C0000E947E0A0E94590B8E010E5F1F4FC12C86
:1023D000D12C7601C39466246A945C2C0E94D52883
:1023E0004B015C012091880530E0A0E1B7E20E943A
:1023F000792E9B01AC01C701B6010E949B2E209152
:102400007F05309180054091810550918205620FD2
:10241000731F841F951F2091BF053091C005409107
:10242000C1055091C205261737074807590718F408
:10243000F801608229C08C2D0E94B20961E070E031
:1024400080E090E00E940429F80110820E94D528C3
:10245000681979098A099B09643F714081059105D2
:1024600040F40E94C809F8019081981778F780839A
:10247000EDCF50FE05C05D9841985E9A409A04C029
:102480005D9A419A5E9840982FEFC21AD20AE20AEA
:10249000F20A0F5F1F4F8FEFC816D104E104F10459
:1024A00009F09BCFCE019395FC01D82E7FEF68EC0D
:1024B0002E2F281B271510F051E056C0DE01129672
:1024C00051E02FEF41E03D91321710F0322F01C063
:1024D000452F5F5F5F3F11F0232FF5CF4193242FEE
:1024E00030E0A1E0B0E0AC0FBD1FA20FB31F5C93C2
:1024F000413079F0DE01A20FB31F5C93423049F006
:10250000AFEFBFEFAC0FBD1FA20FB31F6C934E3FD9
:1025100078F6A2E0B0E0AC0FBD1FA20FB31F7C9312
:102520004D3F30F6A3E0B0E0AC0FBD1FA20FB31FCC
:102530006C93BECF452F242F30E0FC01E20FF31F38
:102540006081AFEFB0E0AC0FBD1FA20FB31F2C91A5
:10255000621748F44150DC01A40FB11D2C91208377
:102560006C934111E8CF5F5F571520F3372D3695F7
:1025700020E0231770F4DC01A20FB11D4C91522F03
:10258000530FFC01E50FF11D50815C9340832E5FDA
:10259000F0CFF9E8EF2EF5E0FF2E8C01802F8D199A
:1025A000871598F4F801C1908F014AE050E06C2D36
:1025B00086EE95E00E94932B6CE286EE95E00E94F9
:1025C0009F2AF701C1927F01E9CF86EE95E00E9434
:1025D000A72A81E0CD5EDE4FEFE00C941F2F1F9203
:1025E0000F920FB60F9211241F932F933F934F9387
:1025F0005F936F937F938F939F93AF93BF93CF938B
:10260000DF93EF93FF93C0918600D0918700809174
:102610008704909188042091A904211155C09E013E
:10262000281B390B8091C3059091C405A091C50565
:10263000B091C60585FD02C036952795253C49E039
:102640003407B8F140910A0150E060E070E02CE1FD
:10265000B695A795979587952A95D1F70097A105E7
:10266000B10521F481E090E0A0E0B0E08417950787
:10267000A607B707D8F480910A018F3FB9F040E070
:1026800080910A01481780F4842F90E0880F991FE9
:10269000FC01E757FB4F20813181FC01E55FFE4FD4
:1026A000318320834F5FECCF1092AA0410920A016D
:1026B0000BC02D3B82E0380720F080910A01803169
:1026C000D8F08FEF80930A01D0938804C0938704D9
:1026D000FF91EF91DF91CF91BF91AF919F918F913A
:1026E0007F916F915F914F913F912F911F910F902B
:1026F0000FBE0F901F90189510910A0181E0810F75
:1027000080930A01C9010E94DE08E12FF0E0EE0F7C
:10271000FF1FE757FB4F91838083D6CF83E08093E1
:1027200080008AE9809381008091C30586FD05C001
:10273000809181008064809381008FEF9FEF909360
:1027400089008093880080916F00806280936F0081
:1027500008950E94300D8091D805843011F41092B4
:10276000D80508956F3018F086958058089589E04F
:10277000689F802D11240895A0E0B0E0E2ECF3E121
:102780000C940A2FC82F0E94E12800913804109160
:10279000390420913A0430913B046B017C01C01A4A
:1027A000D10AE20AF30A9701860149E8C41643E117
:1027B000D406E104F10410F010923C046093380454
:1027C0007093390480933A0490933B042091A904B8
:1027D0008FEF820F8230E8F5E0913C04EE2309F49C
:1027E0006EC1E13011F482E0D8C1E03178F581E0CA
:1027F0008E0F80933C04F0E0E757FB4FC08380319D
:1028000009F0D4C1EBE8F4E0213029F4A181A695C8
:10281000A695808108C080819181A92FA695A69553
:10282000A69596958795A03148F4B0E090E0AA0F60
:10283000BB1FA55FBE4F11969C938E931092AA0466
:10284000329684E0E939F807F9F6B0C110923C04F9
:10285000ADC1233009F023C1E0913C04E11118C05F
:10286000CF3009F011C10E94D5280091B704109112
:10287000B8042091B9043091BA04601B710B820B2B
:10288000930B623071058105910508F089C1FCC088
:10289000E83148F481E08E0F80933C04F0E0E85783
:1028A000FB4FC083F1C0E83109F0ECC0C111EAC0B0
:1028B00040E050E0ABE0CA01B3E0880F991FBA9541
:1028C000E1F7A49F9001A59F300D1124F901E7576E
:1028D000FB4F6081E1817E2F777075956795FC01D4
:1028E000EE0FFF1FE55FFE4F71836083F901E6572E
:1028F000FB4FB081B695B695B695E181FE2FF29566
:10290000FF0FF07E6F2F6B2BE695E695E6957E2FF9
:10291000777075956795FC01EE0FFF1FE35FFE4F23
:1029200071836083F901E557FB4FB081B295B6958D
:10293000B695B370C181DC2FDD0FDD0F6D2F6B2BD2
:10294000C295C695C695C370E281E170EE0FEE0F99
:102950007E2F7C2B75956795FC01EE0FFF1FE15FC5
:10296000FE4F71836083F901E357FB4FB081B69549
:10297000E181FE2FF795FF27F7956F2F6B2BE695DB
:102980007E2F777075956795FC01EE0FFF1FEF5E48
:10299000FE4F71836083F901E257FB4FB081B2951E
:1029A000BF70E181FE2FF295F07F6F2F6B2BE295C8
:1029B000EF707E2F777075956795FC01EE0FFF1F06
:1029C000ED5EFE4F71836083F901E157FB4FB081EB
:1029D000BB1FBB27BB1FC181DC2FDD0F6D2F6B2BF6
:1029E000CC1FCC27CC1FE281E370EE0F7E2F7C2B17
:1029F00075956795FC01EE0FFF1FEB5EFE4F71832F
:102A00006083F901EF56FB4FB081B695B695E18131
:102A1000FE2FF295FF0FFF0FF07C6F2F6B2BE695CB
:102A2000E6957E2F777075956795FC01EE0FFF1F79
:102A3000E95EFE4F71836083F901EE56FB4F208102
:102A40002295269527703181E32FEE0FEE0FEE0FC2
:102A50006E2F622B732F72957695777075956795AB
:102A6000FC01EE0FFF1FE75EFE4F718360834F5F37
:102A70005F4F4230510509F01ECF80919F0483FFC4
:102A80001092AA0410923C040E94D5286093B704C7
:102A90007093B8048093B9049093BA0487C024302B
:102AA00009F084C060913C0461110BC0C83AB1F4D4
:102AB000109279051092780588EA0E94610681E0FB
:102AC0006CC0613019F4C093370404C0623031F433
:102AD000C09336048C2F0E9461065AC0E0913604E0
:102AE0002E2F30E0220F331F462F50E0C9010296EF
:102AF000841795073CF0633268F7FA01EA57FB4FF9
:102B0000C083E8CF2D5F3F4F8C2F90E06091780518
:102B1000709179054217530749F4982F8827862723
:102B20009727909379058093780532C068177907C5
:102B300069F580913704813049F5E13118F080E181
:102B400080933604F0903604CAE8D4E000E010E048
:102B50000F15D0F4FE013197808190E0982F8827DF
:102B60002881822B63E0969587956A95E1F70E940C
:102B7000DE08F801EE0FFF1FE55FFE4F91838083B3
:102B80000F5F1F4F2296E4CF1092AA0410923C04CC
:102B900080913C04882351F08F5F80933C0406C0F1
:102BA00080913C048F5F80933C046ECFCDB7DEB73D
:102BB000E8E00C94262FE82FF0E0E254FA4FE1858C
:102BC000E03150F4F894F0E0EE0FFF1FE55FFE4FA8
:102BD00080819181789408958EE08E0F8B3058F427
:102BE000F0E0E25FF10924E62E9FC0012F9F900DD7
:102BF00011240C960895E03FF1F028F4E03161F0E3
:102C0000E13161F006C0ED3F81F0EE3F89F0E13F38
:102C100049F080E092E0089582E101C083E10E94E2
:102C2000232A089586E090E008958AEF93E00895BE
:102C30008FEF93E0089580E090E00895A2E2B0E085
:102C4000E4E2F6E10C94002F9E012F5F3F4F80E1FC
:102C5000D9011D928A95E9F764E072E086EE95E06D
:102C600029A33AA30E94CD2A0E947C0B1D8A1E8AAA
:102C70001F8A188E312C212C00E0812C912C5401BC
:102C800070E4472E71EE572E7DE9672E78E1772E9E
:102C9000E0E5CE2EE3ECDE2EE12CF12C84EF91E08A
:102CA000A0E0B0E08D8F9E8FAF8FB8A380EC91ED48
:102CB000A8E9BBE1898F9A8FAB8FBC8F80E491EE3E
:102CC000ADE9B8E1898B9A8BAB8BBC8B86EE95E036
:102CD0000E94E12B892B09F4E1C086EE95E00E9469
:102CE0000E2C9C0133272C32310509F442C0ACF480
:102CF0002332310509F0ABC019821A821B821C8273
:102D00001D821E821F82188619861A861B861C86C3
:102D10001D861E861F86188A60C02434310529F05E
:102D20002335310509F4B2C092C064E486EE95E023
:102D30000E949F2A2AE030E040E451EE6DE978E1FC
:102D400086EE95E00E942D2B6CE286EE95E00E94C7
:102D50009F2A2AE030E040EC51ED68E97BE186EE05
:102D600095E00E942D2B6CE286EE95E00E94DF2A12
:102D7000ADCF0F5F043009F0A9CF29813A814B8193
:102D80005C81A8EEB3E00E94882E698B7A8B8B8BD6
:102D90009C8B2D813E814F8158850E94882E698FA2
:102DA0007A8F8B8F9C8F29853A854B855C852D8FFB
:102DB0003E8F4F8F58A32D853E854F8558890E94A1
:102DC000882E6B017C0160323EE47307810591051A
:102DD00030F462E38CE10E949F0900E077CF60331A
:102DE00045E774078105910510F462E2F3CF603482
:102DF0005CE975078105910510F466E2EBCF80E58B
:102E0000C81683ECD806E104F10410F462E1E2CFC5
:102E100090E6C9169AEED906E104F10410F465E1D2
:102E2000D9CFA0E7CA16A1E1DA06A1E0EA06F104CB
:102E300010F461E0CFCFB0EACB16B6E8DB06B1E024
:102E4000EB06F10410F463E0C5CF65E0C3CF10EDED
:102E5000180F1A3008F03ACFE1E0F0E0EC0FFD1F58
:102E600024E0029FE00DF11D112420813181428177
:102E70005381AAE0B0E00E94882E610F711D811D70
:102E8000911D608371838283938320CF49885A8800
:102E90006B887C88812C912C540118CF811491046B
:102EA000A104B10489F4C301B2010E940E0A61E0D9
:102EB00070E080E090E00E9404291D8A1E8A1F8A2B
:102EC000188E312C22242A948D8D9E8DAF8DB8A121
:102ED00088169906AA06BB06D0F40E94C8092D8957
:102EE0003E894F89588D280F311D411D511D2D8B55
:102EF0003E8B4F8B588F381608F4382E821508F405
:102F0000282E3FEF831A930AA30AB30A56C0C301BF
:102F1000B20128EE33E040E050E00E94BF2EBA013B
:102F2000A9012AE030E086EE95E00E94842B6CE255
:102F300086EE95E00E949F2A4AE050E0632D86EEDF
:102F400095E00E94932B6CE286EE95E00E949F2A0A
:102F50006D897E898F89988DA50194010E94BF2E6D
:102F6000BA01A9012AE030E086EE95E00E94842BA8
:102F70006CE286EE95E00E949F2A4AE050E0622DC6
:102F800086EE95E00E94932B6CE286EE95E00E941F
:102F9000DF2A4C0C5D1C6E1C7F1C898D9A8DAB8DBD
:102FA000BC8D84159505A605B70520F449885A8877
:102FB0006B887C88812C912C540129893A894B8912
:102FC0005C89283E33404105510509F07FCEA29629
:102FD000E2E10C941C2FACE1B0E0E1EFF7E10C94DE
:102FE0000A2F0E94E1286B017C0181E00E947E0A89
:102FF00014E703E0198361E0CE0101960E94DB0B28
:10300000009377050E94590B6AEF70E080E090E032
:103010000E94042980917705833089F486EE95E03B
:103020000E94E12B892B59F40E94E1286C197D093B
:103030008E099F096038734C894C9140D8F2809179
:103040007705833009F44FC08FE70E9477090E940B
:103050008A098983843511F083E05CC00E948A0963
:1030600010924A0580934B050E948A0920914A05D7
:1030700030914B05280F311D30934B0520934A05A5
:103080000E948A0980934C050E948A0980934D050D
:10309000813110F7F12C0F2D10E080914D0590E05B
:1030A000880F991F0817190740F40E948A09F80130
:1030B000E25BFA4F8083F394EECF80E7898361E08F
:1030C000CE0101960E94DB0B83E0809377050E947E
:1030D000590B62E370E080E090E00E940429809147
:1030E0007705833011F482E015C08FE70E947709DD
:1030F0000E948A098983803509F0AECF03EA15E082
:103100000E948A09F80181938F01F5E00E3B1F07A9
:10311000B9F781E06C96E8E00C94262F8091490580
:10312000992787FD9095A92FB92FFC013196EB3097
:10313000F10508F066C0EC5CFF4F0C94372F62E796
:1031400078E086EE95E00E94BB2A88E893E00E9432
:10315000300C6AE578E086EE95E00E94BB2A65E3D4
:1031600078E086EE95E00E94BB2A6BE078E086EE80
:1031700095E00E94BB2A6AEE77E086EE95E00E9419
:10318000BB2A6DEB77E086EE95E00E94BB2A67E9EB
:1031900077E086EE95E00E94BB2A63E777E086EE53
:1031A00095E00E94BB2A6CE477E086EE95E00E94F1
:1031B000BB2A86EE95E00E94A72A0E94700D21C0CE
:1031C0006FE277E01AC06AE077E017C065EF76E05B
:1031D00014C066ED76E011C062E976E00EC06DE7DE
:1031E00076E00BC068E676E086EE95E00E94BB2AAA
:1031F00062E276E002C06CE076E086EE95E00E9446
:10320000BB2A6AE070E080E090E00E94042986EE2C
:1032100095E00E94E12B892B29F086EE95E00E9433
:103220000E2CF5CF0895ACE1B0E0E9E1F9E10C94A2
:103230000A2F909149059F3F09F023C1482F50E084
:10324000FA013A97EF36F10508F00FC1E15CFF4F44
:103250000C94372F61E172E0A0C06DE172E086EE60
:1032600095E00E94CD2A85E789838BE1E3EAF5E0CA
:10327000DE01129601900D928A95E1F76CE1CE0184
:1032800001960E94DB0B0E94590B83E08093770527
:1032900068EC70E080E090E00E940429809177055E
:1032A000843009F0E2C08FE70E9477090E948A0902
:1032B0008983853509F0D9C06DEE74E086EE95E01E
:1032C0000E94BB2A6FEC74E086EE95E00E94BB2A58
:1032D00061EB74E096C065E372E086EE95E00E94D3
:1032E000CD2A89E6898361E0CE0101960E94DB0B3D
:1032F0000E94590B83E08093770568EC70E080E0D2
:1033000090E00E94042980917705843009F0ADC0D7
:103310008FE70E9477090E948A0989838E010E5FD8
:103320001F4F7E014DE1E40EF11C0E948A09F80155
:1033300081938F01EE15FF05C1F78BE1FE013296F7
:10334000A3EAB5E001900D928A95E1F7898189346D
:1033500009F08BC063E974E086EE95E00E94BB2A19
:1033600065E774E086EE95E00E94BB2A67E574E0AD
:1033700048C06FE472E086EE95E00E94CD2A8EEFA1
:103380008093490572C080528750805390914C05BC
:10339000981708F066C06EE572E086EE95E00E9430
:1033A000CD2A63C084E18093490560E274E029C0BE
:1033B00085E18093490569EE73E023C086E180933F
:1033C000490562EB73E01DC087E18093490568E61B
:1033D00073E017C088E18093490567E573E011C089
:1033E00089E18093490563E473E00BC08AE180932F
:1033F00049056EE273E005C08BE18093490566E004
:1034000073E086EE95E00E94BB2A2FC06CEE72E05E
:1034100086EE95E00E94BB2A8091B10591E01DC027
:1034200066ED72E086EE95E00E94BB2A8091B105C0
:1034300092E013C061EC72E086EE95E00E94BB2A38
:103440008091B10594E009C066EA72E086EE95E0ED
:103450000E94BB2A8091B10598E089278093B1052D
:103460008FEF809349050E94111086EE95E00E942F
:10347000E12B892B09F45BC186EE95E00E940E2CAE
:10348000F4CF0E941011882309F451C18091E30404
:10349000811104C08FEF8093490541C140E050E0A5
:1034A00060E070E084EE94E00E94AE2F4091490508
:1034B000042F112707FD1095212F312FF801319787
:1034C000EB31F10508F01BC1E255FF4F0C94372F8B
:1034D000552747FD509520914C0530E024173507BE
:1034E0000CF40DC18B019C01015011092109310916
:1034F000003211052105310558F0C0904D05EFE46B
:10350000F5E0F12CD12CA8E2EA2E415051090FC070
:10351000FA01ED55FA4F61506083D9C0DF01119770
:103520002C9130E02417350729F0F3943296FC10E3
:10353000F5CFCBC00E2D10E020E030E006171707C6
:103540002807390741F42081DA01AD55BA4F1196A9
:103550002C93DD24D394E394E8CF6F3F710581056C
:10356000910511F008F0CBC06093BB05B0C06F3F70
:1035700071058105910511F008F0C1C06093BC058B
:10358000A6C06F3F71058105910511F008F0B7C025
:103590006093BD059CC02091E40420622037E9F4CB
:1035A00040E050E060E070E085EE94E00E94AE2FD5
:1035B0009B01AC01DC01CB010197A109B10908977E
:1035C000A105B10508F0AEC0A4EDB0E30E94882EBD
:1035D0006A5E7C4A8A46954E24C02636E9F440E06D
:1035E00050E060E070E085EE94E00E94AE2F9B0119
:1035F000AC01DC01CB010197A109B1090797A10535
:10360000B10508F08FC0A8EAB1E60E94882E645E7A
:103610007C438E46944E05C0611571058105910568
:1036200079F08B019C010054114E2D49384101382D
:10363000F0EF1F07FAEF2F07F2E03F0708F05FC037
:103640006093B3057093B4058093B5059093B60568
:103650003EC06F3F71058105910511F008F04FC024
:103660006093B70534C08B019C01015011092109F9
:1036700031090F3F11052105310508F040C0609365
:10368000B80525C08B019C01045C19402109310952
:103690000D344DE114072105310528F47093BA0566
:1036A0006093B90514C0611571058105910521F478
:1036B0008FEF8093B2050BC06134710581059105D0
:1036C000F0F461506093B20502C0DD20C1F080913A
:1036D000E20481111AC08091830590918405A09124
:1036E0008505B09186050196A11DB11D80938305C6
:1036F00090938405A0938505B093860506C060E786
:1037000072E086EE95E00E94CD2A0E9406118FEFAE
:10371000809349056AE086EE95E00E94DF2A0E94C8
:10372000111005C061E070E080E090E07ACF6C9607
:10373000E8E00C94262F6AE572E086EE95E00E94A0
:10374000BB2A62E472E086EE95E00E94BB2A86EE18
:1037500095E00E94E12B892B31F086EE95E00E94E6
:103760000E2C0E9413190E94EB17823029F083302F
:1037700051F46DE072E002C064E272E086EE95E022
:103780000E94BB2A08958FEF809349051092E204AE
:103790000E941110809149058E3F69F086EE95E0F8
:1037A0000E94E12B892BB1F386EE95E00E940E2C4E
:1037B0000E941319EFCF08950F931F93109149059D
:1037C0001F3F09F0D2C0893409F457C000F588338F
:1037D00009F469C058F4803309F477C008F061C077
:1037E0008B3109F440C08132B1F1B9C0813409F4A0
:1037F00087C030F4893309F466C0803461F1AFC00A
:10380000823409F48EC0863409F448C0A8C08236D8
:1038100009F487C078F4883531F128F48235C1F194
:103820008335E1F09CC08A3509F494C0813609F4EF
:1038300067C095C0823761F128F4863679F1893600
:10384000E1F08DC0883779F08A3709F483C0833777
:1038500009F085C003C061E172E015C00E94410D0E
:103860006EE872E004C00E944A0D68EA72E086EEDB
:1038700095E00E94CD2A8EEF70C00E947A060E94C9
:10388000BF0667EC72E086EE95E00E94CD2A67C025
:1038900081E00E94DF0660EE72E0F5CF0E94BB106F
:1038A0005EC080535AC06AEF71E086EE95E00E94D8
:1038B000BB2A9091A20588E0890F8871977E892B99
:1038C0008093A2051AC089E048C067EE71E086EED9
:1038D00095E00E94BB2A8091C3059091C405A091F8
:1038E000C505B091C60520E182278093C30590935A
:1038F000C405A093C505B093C605109349052FC014
:1039000061ED71E086EE95E00E94BB2A8091C305CF
:103910009091C405A091C505B091C60540E48427E7
:1039200010C060EC71E086EE95E00E94BB2A8091A9
:10393000C3059091C405A091C505B091C60520E2CC
:1039400082278093C3059093C405A093C505B093C7
:10395000C60502C00E949B1B8FEF80934905809192
:1039600049058E3F09F0D4C0DDC00E9410118823A4
:1039700009F4D8C08091E304811104C08FEF8093D3
:103980004905C6C040E050E060E070E084EE94E09D
:103990000E94AE2F00914905112707FD1095212F98
:1039A000312FF8013197E930F10508F0B4C0E75341
:1039B000FF4F0C94372F8B019C010154114E2D4960
:1039C00038410F37104F2A4F324008F0A4C060939F
:1039D0007F0570938005809381059093820577C061
:1039E0006093830570938405809385059093860585
:1039F00081E08093E2046BC0683071058105910518
:103A000008F089C06093870562C08B019C0101505A
:103A10001109210931090A3011052105310508F084
:103A20007AC06093880553C061EB71E084EE94E046
:103A30000E94E83010E0009799F00E94C230009791
:103A400079F0183130F4E12FF0E0E658FA4F87872B
:103A50001F5F61EB71E080E090E00E94E830EBCF07
:103A60001831A8F5E12FF0E0E658FA4F17861F5FEE
:103A7000F7CF653071058105910508F04CC0609362
:103A8000A10525C08B019C010150110921093109B3
:103A90000630110521053105F0F52091A205287F9A
:103AA000262B2093A20513C08B019C010150110904
:103AB000210931090115124C2140310560F560934F
:103AC0007B0570937C0580937D0590937E058091A6
:103AD000E204811113C08091830590918405A09127
:103AE0008505B09186050196A11DB11D80938305C2
:103AF00090938405A0938505B09386050E940611D6
:103B00008FEF809349056AE086EE95E00E94DF2AF8
:103B10000E948E1807C060E772E086EE95E00E9472
:103B2000CD2AECCF1F910F9108958FEF8093490517
:103B30001092E2040E948E18809149058E3F69F030
:103B400086EE95E00E94E12B892BB1F386EE95E09D
:103B50000E940E2C0E94DC1BEFCF6AE070E080E038
:103B600090E00E94042986EE95E00E94E12B892BCB
:103B700029F086EE95E00E940E2CF5CF0895CF93A4
:103B8000C82F682F86EE95E00E943B2C90916E0521
:103B90009C2790936E05CF910895A1E0B0E0E3EDEE
:103BA000FDE10C94102F99830E94BF1D9981892FEC
:103BB0000E94BF1D2196E2E00C942C2F1F93CF93FF
:103BC000DF93182FEB0110926E0565EB70E086EE27
:103BD00095E00E94590662E670E086EE95E00E944C
:103BE0005906812F0E94BF1DCE010E94CD1DDF917D
:103BF000CF911F91089560916E0586EE95E00E9429
:103C00003B2C0895A1E2B0E0E8E0FEE10C940C2F1B
:103C10007B018A018C3009F452C108F040C0863023
:103C200009F4BCC018F5833009F491C070F48130F8
:103C300009F472C0823009F049C26BE170E082E0A1
:103C40000E94DE1D03EA15E078C0843009F487C0C5
:103C5000853009F03BC260914D0570E0660F771F1B
:103C600085E00E94DE1D0EE415E086C0893009F46F
:103C7000A7C070F4873009F49BC0883009F026C2D1
:103C800061E070E088E00E94DE1D8091D80524C2CA
:103C90008A3009F4CAC08B3009F4F1C017C28A36E1
:103CA00009F474C1D8F4873609F439C138F485367B
:103CB00009F40DC1863609F41EC108C2883609F41C
:103CC00036C1893609F002C261E070E089E60E94DF
:103CD000DE1D0E947A060E94BF06F6C18D3609F4E9
:103CE000D3C138F48B3609F490C18C3609F499C1EC
:103CF000EDC18E3609F4DDC1873C09F0E7C161E012
:103D000070E087EC0E94DE1D81E00E94BF1D0E94D2
:103D1000FB1D10926F05E4C169E270E081E00E9432
:103D2000DE1D0AE715E0F80181918F010E94BF1D99
:103D3000F5E0033A1F07B9F7D1C1F80181918F016E
:103D40000E94BF1DF5E00E3B1F07B9F7C7C161E038
:103D500070E083E00E94DE1D0E94EB17BDC161E0B0
:103D600070E084E00E94DE1D81E00E94BF1D0E9481
:103D7000FB1D0E941E16B4C180914D0590E0880F76
:103D8000991F98012E5435402817390708F0A6C10D
:103D9000F80181918F010E94BF1DEECF62E070E0BB
:103DA00086E00E94DE1D88E893E00E94CD1D96C14A
:103DB00061E070E087E00E94DE1D80914C058CC1BF
:103DC00086E6898361E0CE0101960E94DB0B0E94AA
:103DD000590B83E08093770568EC70E080E090E019
:103DE0000E940429809177058430D9F48FE70E94DE
:103DF00077090E948A098983863469F460E270E059
:103E000089E00E94DE1D10E20E948A090E94BF1D07
:103E10001150D1F763C161E070E089E00E94DE1DBE
:103E200053C161E070E089E054C169E170E08AE06B
:103E30000E94DE1D1092BE05209176058091C3057B
:103E40009091C405A091C505B091C605222311F03B
:103E5000806801C08F778093C3059093C405A093B9
:103E6000C505B093C6050EEB15E0F80181918F01F1
:103E70000E94BF1DF5E0073D1F07B9F72FC161E2A2
:103E800070E08BE00E94DE1D8091AA048F3F39F024
:103E90008091AA0491E0980F9093AA0402C08091A7
:103EA000AA040E94BF1D10E0812F0E94DB150E9412
:103EB00009090E94CD1D1F5F1031B1F70FC161E0EC
:103EC00070E08CE00E94DE1D8091D70505C161E0A5
:103ED00070E085E60E94DE1D89E2E816F10409F033
:103EE000FAC0D801EAE7F5E08D91819385E0E33AE5
:103EF000F807D1F7E9C061E070E086E60E94DE1DB8
:103F0000EBE1EE16F10409F0E6C0D801E3EAF5E0D2
:103F10008D91819385E0EE3BF807D1F7D5C061E044
:103F200070E087E60E94DE1D0E94410DCDC061E079
:103F300070E088E60E94DE1D85E789838BE1E3EA75
:103F4000F5E0DE01129601900D928A95E1F76CE1A1
:103F5000CE0101960E94DB0B0E94590B83E08093F7
:103F6000770560E273E080E090E00E940429809190
:103F70007705843009F0AFC08FE70E9477090E946F
:103F80008A098983853509F0A6C09EC061E070E08A
:103F90008AE60E94DE1D89E6898361E0CE010196F2
:103FA0000E94DB0B0E94590B83E08093770560E24F
:103FB00073E080E090E00E940429809177058430CE
:103FC00009F089C08FE70E9477090E948A098983D6
:103FD0008E010E5F1F4F7E01EDE1EE0EF11C0E947F
:103FE0008A09F80181938F01EE15FF05C1F78BE176
:103FF000FE013296A3EAB5E001900D928A95E1F7B1
:104000008981893409F067C05FC061E070E08BE6A8
:104010000E94DE1DF80180818093D8050E944A0D20
:1040200053C061E070E08CE60E94DE1DF0E2EF1606
:10403000F10461F487E6898380E2F801DE011296DB
:1040400001900D928A95E1F761E203C087E48983CC
:1040500061E0CE0101960E94DB0B0E94590B83E0C8
:10406000809377056CE474E080E090E00E9404297E
:1040700080917705843079F58FE70E9477090E9457
:104080008A09873441F520C061E070E08DE60E9426
:10409000DE1D89E1E816F104F1F4D801EEEBF5E05C
:1040A0008D91819385E0E73DF807D1F70E948E134B
:1040B0000BC061E070E08EE60E94DE1DF801808199
:1040C0008093D7050E942B0D81E006C061E070E06F
:1040D0008AEC0E94DE1D80E00E94BF1D0E94FB1D35
:1040E000A196E6E00C94282FA0E0B0E0EAE7F0E229
:1040F0000C940A2FCAECD3E014E606E035E0F32E68
:1041000044E0E42E53E0D52E62E0C62E86EE95E024
:104110000E94E12B892B09F49BC086EE95E00E945A
:104120000E2C282F809335044091340450E0473002
:10413000510560F7FA01EE52FF4F0C94372F853B83
:1041400029F781E080933404E1CF823609F07DC005
:10415000C0923404DBCF8093330480933204D09236
:104160003404D4CF9C01332730933104209330049E
:1041700090913204982790933204E0923404C6CF91
:10418000382F22274091300450913104242B352BB5
:104190003093310420933004909132049827909307
:1041A0003204F09234042536310508F4AFCF61E0D3
:1041B00070E08CEC0E94DE1D81E00E94BF1D0E9419
:1041C000FB1D43C020912E0430912F04F901E653CA
:1041D000FC4F808390913204982790933204C90158
:1041E000019690932F0480932E04209130043091F7
:1041F00031048217930708F489CF0093340486CFE3
:104200008091320482130BC060912E0470912F04B0
:104210004AEC53E0809133040E94021E0DC062E01C
:1042200070E08BEC0E94DE1D809133040E94BF1D64
:1042300080916E050E94BF1DFE01812F11928A950B
:10424000E9F710922F0410922E04109234045ECFDE
:10425000CDB7DEB7E8E00C94262F81E080936F05A0
:1042600080916F05882349F086EE95E00E94E12B4E
:10427000892BB1F30E947420F3CF0895AAE2B0E035
:10428000E4E4F1E20C94082F0E94D5286B017C0134
:1042900081E00E947E0A86EE95E00E94E12B892B48
:1042A00029F086EE95E00E940E2CF5CF5E9840989E
:1042B00011E072E6B72EE9E2AE2E03E00E94D528A7
:1042C0006C197D098E099F09693C7105810591056D
:1042D000E0F11123D1F10E94D5286B017C015D9A98
:1042E000419A80ED97E00E94A807B982EAE7F5E0DD
:1042F000DE0112968A2D01900D928A95E1F76AE20D
:10430000CE0101960E94DB0B5D98419880E090E021
:104310000E94A807009377050E94590B62E370E0A2
:1043200080E090E00E94042980917705843061F458
:10433000009377058FE70E9477090E948A0911E0B0
:10434000823419F410E001C011E083E10E94FA29DF
:10435000892BA1F411E012C05E9A409A5D9A419AAD
:1043600086EE95E00E940E2C8D309105B9F06CF42C
:104370000A97A1F05E9840985D98419886EE95E086
:104380000E94E12B892B41F799CF8332910579F077
:104390008234910579F70E942D21ECCF62EB71E018
:1043A00086EE95E00E94BB2A0E94951DE3CF0E94F5
:1043B0001E16E0CF8F929F92AF92BF92CF92DF9264
:1043C000EF92FF921F93CF93DF9383E10E94FA292C
:1043D000892B09F089C068EC70E080E090E00E94D1
:1043E000042980E090E00E94A8070E94D5284B0194
:1043F0005C016B017C0180ECC80E82E1D81EE11CDF
:10440000F11C0E94D5286C157D058E059F0530F4A2
:1044100083E10E94FA29892BA1F364C083E10E9401
:10442000FA29892B09F05EC080ED97E00E94A80769
:104430000E94D5286B017C01D0E0C1E088E4880EA1
:1044400086E2981EA11CB11C11E083E10E94FA29AA
:10445000892B21F58C149D04AE04BF0430F480ED4B
:1044600097E00E94A807D1E0F0CF0E94D5286C19F0
:104470007D098E099F09693C71058105910528F325
:104480000E94D5286B017C01C12719F080ED97E0CF
:1044900002C080E090E00E94A807D7CF80E090E0C3
:1044A0000E94A807DD23B9F08091D70590E001961E
:1044B00065E070E00E94AB2E8093D7050E942B0D23
:1044C0000E94A9130E944A0D64EF71E080E090E021
:1044D0000E94042909C080E00E94DF060E94C211E8
:1044E0000E94410D0E943E21DF91CF911F91FF90CC
:1044F000EF90DF90CF90BF90AF909F908F900895F6
:10450000CF92DF92EF92FF9280E00E94DA070E9442
:10451000B10761E086E00E948E2961E085E00E949B
:104520008E2961E08EE00E948E2961E08FE00E947A
:104530008E2960E083E10E948E2960E088E00E947D
:104540008E2961E088E00E94C7290E949F0740E011
:1045500052EC61E070E086EE95E00E94292D0E9409
:10456000A9130E944A0D0E948E138FEF8093AA0414
:104570000E94C60778940E94D5286B017C01809127
:10458000AA048F3F59F40E94D5286C197D098E0921
:104590009F09603D77408105910588F380ED97E0A4
:1045A0000E94A80761E083E10E94C7295E9A409AB1
:1045B00086EE95E00E94E12B892B29F086EE95E0AE
:1045C0000E940E2CF5CF6DEF72E086EE95E00E9412
:1045D0009C2A88E893E00E94300C64E173E086EE48
:1045E00095E00E949C2A4AE050E069E070E086EE87
:1045F00095E00E946C2B62E370E080E090E00E9406
:10460000042986EE95E00E94E12B04970CF186EEDA
:1046100095E00E940E2C82349105D1F486EE95E04F
:104620000E940E2C8E34910599F486EE95E00E943E
:104630000E2C8434910561F486EE95E00E940E2CD8
:10464000819731F480E090E00E94A8070E943E210B
:1046500040917B0550917C0560917D0570917E05B0
:10466000DB01CA010197A109B1090497A105B105B0
:1046700090F44093A904433051F42EE240EA56E806
:1046800061E070E086EE95E00E94AA2D08C040E04F
:1046900052EC61E070E086EE95E00E94292D0E94C8
:1046A000DA215E98409880E090E00E94A8070E947E
:1046B0008E131092C9048091C30583FF11C08091AD
:1046C0008F05882351F080919605882331F08091E1
:1046D0009D05882311F087E001C085E08093C9041F
:1046E00080E00E947E0A8091CA040E94B2090E9462
:1046F000590B10923F0410923E0410923D04F12C8D
:104700008091D8058F15B0F062E370E080E090E012
:104710000E94042980ED97E00E94A80762E370E000
:1047200080E090E00E94042980E090E00E94A807C9
:10473000F394E6CF8091A20584FF08C0982F98716A
:1047400081E0983109F080E00E947E118FE00E94A4
:10475000DA07FF90EF90DF90CF900895EF92FF92ED
:104760000F931F93CF93DF938C016EE770E086EE7B
:1047700095E00E945906E801F12CF0E2EF2E8E013F
:1047800088818D57823048F46DE770E086EE95E0C1
:104790000E94590688818E2588832196F8016081C0
:1047A00086EE95E00E943B2CF394F9E0FF12E7CFF0
:1047B0006EE770E086EE95E00E945906CDB7DEB751
:1047C000E6E00C94282FA9E0B0E0E9EEF3E20C94C7
:1047D000102F9091CB0491110EC09EEF99838A8384
:1047E0006B8350E0559547954C832D831986188629
:1047F0001F821E822EC04091D004842F90E0B4E02E
:1048000095958795BA95E1F7242F2F7030E08217A0
:10481000930719F18DEF89831B82FE01349650E0D6
:10482000842F90E0A4E095958795AA95E1F7242F31
:104830002F7030E08217930749F0DC01AF52BB4F75
:104840008C918193405F5F5F563051F74093D00465
:104850005A83CE0101960E94AE238091CB0490E052
:10486000019666E070E00E94AB2E8093CB042996FF
:10487000E2E00C942C2FA0E0B0E0E1E4F4E20C9430
:10488000092F6C016EE770E086EE95E00E945906F4
:104890008601E12CF12CC0E0D0E030E2B32EF8012B
:1048A000608183E8860F823078F46DE770E086EEF1
:1048B00095E00E945906F80160816B2570E086EE54
:1048C00095E00E94590604C086EE95E00E943B2CBC
:1048D000E114F10459F0F80180819E01280F311D87
:1048E000C901C92FDD27C80FD91FDD273FEFE31A04
:1048F000F30A89E0E816F10459F028E0E216F10421
:1049000021F48C2F8095F60180870F5F1F4FC7CF52
:10491000CDB7DEB7E9E00C94252FA9E0B0E0E3E9DC
:10492000F4E20C94102FE82F362F8091CB0490E006
:10493000019664E270E00E94AB2E8093CB0458E9AC
:10494000598350E15A83813089F048F08230B9F0C0
:104950008330D9F48B8381EF8C833D8319C085E04C
:104960008B8381EF8C832F5F2D8312C08B8381EF2C
:104970008C8384E6489FA00111245D8309C084E0F4
:104980008B8381EF8C83ED8303C00E94BB1104C035
:10499000CE0101960E943B242996E2E00C942C2F34
:1049A000A2E0B0E0E6EDF4E20C94052F182F762E8D
:1049B0002A8349830E94E1286B017C018091E104F4
:1049C0008090CC049090CD04A090CE04B090CF0401
:1049D0002A8149818823C1F0D701C6018819990924
:1049E000AA09BB094C015D0191EE89169EE2990668
:1049F000A104B10420F1241708F4422F202F672DC1
:104A0000812F0E948D2413C0D701C60188199909EE
:104A1000AA09BB094C015D0191E3891695E7990646
:104A2000A104B10460F0672D812F0E94E323C0929E
:104A3000CC04D092CD04E092CE04F092CF04229622
:104A4000EDE00C94212FA2E2B0E0E9E2F5E20C9453
:104A5000062F8CE00E94990981110FC06CE173E070
:104A600086EE95E00E94CD2A5E9A409A80E00E94F0
:104A70007E0A0E94590B5E98409886EE95E00E944F
:104A8000E12B892B01F186EE95E00E940E2C90918E
:104A9000A904992319F00E94BC13EFCF40913E0462
:104AA00050E09A012F5F3F4F2F71332760913F04F1
:104AB00070E02617370709F3FA01E75BFB4F8083A5
:104AC00020933E04DACF80917705843009F086C0C8
:104AD0000E94E128611571058105910549F06093F7
:104AE000BB047093BC048093BD049093BE040CC0BF
:104AF00081E090E0A0E0B0E08093BB049093BC0420
:104B0000A093BD04B093BE048091AD049091AE0417
:104B100081609093AE048093AD0483E08093770529
:104B20008FE70E94770909E614E00E948A09F801DC
:104B300081938F01F4E002371F07B9F720917204C7
:104B400080916904982F922796FF3BC090E49227AA
:104B500090937204982F98739833F1F410E0212FFA
:104B600030E080916904877090E0821793074CF1E0
:104B70001F5F2091A205812F90E0FC01E759FB4FB8
:104B800024FF04C080810E949D11E9CF608186EEE0
:104B900095E00E943B2CE3CF8F7399F480916A04D7
:104BA0008093B60480916B048093B40480916C046C
:104BB0008093B30480916F0490E09093AC04809351
:104BC000AB0480913D04813019F482E080933D0470
:104BD00080913D04833011F410923D040E94E1283D
:104BE0006B017C018091AF049091B004A091B1045D
:104BF000B091B2040097A105B105C9F0A7019601D3
:104C0000281B390B4A0B5B0BDA01C901883B9B401F
:104C1000A105B10560F00E94C8098093B504109207
:104C2000AF041092B0041092B1041092B2048091BB
:104C3000BF049091C004A091C104B091C204460188
:104C40005701881A990AAA0ABB0A8AE795E00E94C6
:104C5000F40786169706A806B90608F4A9C0C092FC
:104C6000BF04D092C004E092C104F092C2040E943A
:104C700057068091AA048830A0F08091C3059091D6
:104C8000C405A091C505B091C6055CE1B695A79590
:104C9000979587955A95D1F7892B8A2B8B2B09F0FD
:104CA000AEC18091AA048F5F8093AA048091BB0457
:104CB0009091BC04A091BD04B091BE040097A105E1
:104CC000B105F1F0C81AD90AEA0AFB0A8AE795E0A9
:104CD0000E94F4076C157D058E059F0508F014C130
:104CE0008091C30584FD04C080ED97E00E94A80771
:104CF0001092BB041092BC041092BD041092BE042A
:104D000090917204907C9093720450913E04809133
:104D10003F0420913D04581709F413C1223009F0D3
:104D200010C1905890937204E091A205E770F0E0F2
:104D3000E658FC4F6081693008F0EBC0615040E0FC
:104D40004613E9C080933F0487E3840F9091720477
:104D5000892B809372044093400483E080933D0448
:104D60005D9A419A809187059091C904911138C14B
:104D70000E94790A8091CA040E94B209E091A205BA
:104D8000E770F0E0E658FC4F608182E794E00E9413
:104D9000940BE091CA04EF5FE093CA04E83109F490
:104DA0002BC1F0E0E658FA4F8785882309F424C127
:104DB0000E94030C813069F58091A205887149F148
:104DC0008091AD049091AE04880F991F9093AE042A
:104DD0008093AD0483E0809377050E94590B0E9475
:104DE000E1286093AF047093B0048093B104909372
:104DF000B204672B682B692B61F481E090E0A0E09E
:104E0000B0E08093AF049093B004A093B104B0934A
:104E1000B2048091A20584FF2BC08091BB049091C5
:104E2000BC04A091BD04B091BE04892B8A2B8B2BAE
:104E3000F9F08091AD049091AE048E7F0E942A0912
:104E4000182F6091AB048091B6040E94B213482FD2
:104E5000612F8091B50449A30E94B2130091D80537
:104E6000282F49A16091B3048091B4040E94D024FA
:104E70005D9841988091C7048130C1F018F082306C
:104E8000B1F1CBC083E10E94FA29892B09F0C5C09A
:104E900081E08093C7040E94D5286093C304709377
:104EA000C4048093C5049093C604B7C083E10E94F4
:104EB000FA29892B31F50E94D528C090C304D090DF
:104EC000C404E090C504F090C6046C197D098E09F5
:104ED0009F09693E73408105910508F49EC082E0F8
:104EE0008093C70480ED97E00E94A80796C083E1F5
:104EF0000E94FA29892B09F490C080E090E00E947A
:104F0000A8071092C70489C080E090E00E94A8071B
:104F1000F7CE68E014CF851709F414CF4F5F242F24
:104F200030E090E0F901EE58FB4FDC01A75BBB4F8E
:104F30007C917083F901E05CFB4F708301968F7167
:104F4000FFCE2430B1F42091400481E494E0A3E743
:104F5000B4E0FC013E2F381B321718F431913D9319
:104F6000F9CF87E3820F90917204892B80937204AA
:104F7000F4CE8091C704823059F49160909372040A
:104F80005E9A409A8E010F5F1F4FF12CB80111C03D
:104F90005E98409880913D04811103C081E0809328
:104FA0003D0480913D04833069F784E080933D04A3
:104FB000E9CF8F2D69A37AA30E94DB15F8018193B5
:104FC00091938F01F39469A17AA1F0E1FF12F1CFDF
:104FD0008091A20543E754E087700E947908C0CE13
:104FE000882309F4C5CE2091C80431E0320F3093F4
:104FF000C8042913BDCE0DC01092CA04D9CE809129
:10500000AA04883011F45E9A409A89E08093AA0439
:10501000CFCE1092C8048150ABCEA296ECE00C9497
:10502000222F8230E8F4E82FF0E0EE0FFF1FE75266
:10503000FA4F71836083813041F0809169008C7FE9
:10504000842B80936900E89A089580916900440F49
:10505000551F440F551F837F842B80936900E99A65
:1050600008951F920F920FB60F9211242F933F9322
:105070004F935F936F937F938F939F93AF93BF9360
:10508000EF93FF938091D9059091DA05892B29F050
:10509000E091D905F091DA050995FF91EF91BF9163
:1050A000AF919F918F917F916F915F914F913F91C0
:1050B0002F910F900FBE0F901F9018951F920F9277
:1050C0000FB60F9211242F933F934F935F936F93DB
:1050D0007F938F939F93AF93BF93EF93FF938091B1
:1050E000DB059091DC05892B29F0E091DB05F0913F
:1050F000DC050995FF91EF91BF91AF919F918F9141
:105100007F916F915F914F913F912F910F900FBEC3
:105110000F901F9018951F920F920FB60F921124A7
:105120002F933F938F939F93AF93BF938091DE050F
:105130009091DF05A091E005B091E1053091DD058A
:1051400023E0230F2D3720F40196A11DB11D05C0CA
:1051500026E8230F0296A11DB11D2093DD05809343
:10516000DE059093DF05A093E005B093E105809103
:10517000E2059091E305A091E405B091E505019663
:10518000A11DB11D8093E2059093E305A093E40572
:10519000B093E505BF91AF919F918F913F912F9172
:1051A0000F900FBE0F901F9018952FB7F894609135
:1051B000DE057091DF058091E0059091E1052FBF3C
:1051C00008953FB7F8948091E2059091E305A0918E
:1051D000E405B091E50526B5A89B05C02F3F19F061
:1051E0000196A11DB11D3FBF6627782F892F9A2FE9
:1051F000620F711D811D911D42E0660F771F881F90
:10520000991F4A95D1F70895CF92DF92EF92FF92BE
:10521000CF93DF936B017C010E94E128EB01C11465
:10522000D104E104F10479F00E94E1286C1B7D0BAC
:10523000683E7340A0F381E0C81AD108E108F10884
:10524000C851DC4FECCFDF91CF91FF90EF90DF9012
:10525000CF900895789484B5826084BD84B58160D0
:1052600084BD85B5826085BD85B5816085BDEEE66E
:10527000F0E0808181608083E1E8F0E0108280814D
:1052800082608083808181608083E0E8F0E08081BB
:1052900081608083E1EBF0E0808184608083E0EBDB
:1052A000F0E0808181608083EAE7F0E080818460C3
:1052B000808380818260808380818160808380811F
:1052C000806880831092C1000895833081F028F4B3
:1052D000813099F08230A1F008958630A9F08730AE
:1052E000B9F08430D1F4809180008F7D03C080912B
:1052F00080008F7780938000089584B58F7702C0F7
:1053000084B58F7D84BD08958091B0008F7703C0F0
:105310008091B0008F7D8093B0000895CF93DF938C
:1053200090E0FC01ED50F44F2491FC01E95FF34F54
:105330008491882349F190E0880F991FFC01E15D79
:10534000F34FA591B4918B5D934FFC01C591D4911E
:105350009FB7611108C0F8948C91209582238C939B
:10536000888182230AC0623051F4F8948C91322FE4
:10537000309583238C938881822B888304C0F89492
:105380008C91822B8C939FBFDF91CF910895A1E0E8
:10539000B0E0EDECF9E20C940E2F282F30E0F9018B
:1053A000E152F44F8491F901ED50F44F1491F90159
:1053B000E95FF34F04910023C9F0882321F069834A
:1053C0000E9465296981E02FF0E0EE0FFF1FEB5D81
:1053D000F34FA591B4919FB7F8948C91611103C0DC
:1053E0001095812301C0812B8C939FBF2196E4E00F
:1053F0000C942A2FCF93DF93282F30E0F901E1524C
:10540000F44F8491F901ED50F44FD491F901E95F23
:10541000F34FC491CC2391F081110E946529EC2FA8
:10542000F0E0EE0FFF1FE55EF34FA591B4912C91D4
:105430002D2381E090E021F480E002C080E090E044
:10544000DF91CF9108958E3008F08E5087702091B3
:105450009D0190E4299F90011124822B80937C0070
:1054600080917A00806480937A0080917A0086FD32
:10547000FCCF809178002091790090E0922B0895E4
:10548000A0E0B0E0E6E4FAE20C940A2F6C017A01A5
:10549000EB01E60EF71E00E010E0CE15DF0561F02F
:1054A0006991D601ED91FC910190F081E02DC6014A
:1054B0000995080F191FF1CFC801CDB7DEB7E8E095
:1054C0000C94262F6115710589F0DB010D900020E9
:1054D000E9F7AD0141505109461B570BDC01ED9135
:1054E000FC910280F381E02D0995089580E090E021
:1054F0000895EF92FF920F931F93CF93DF938C0148
:10550000FB01C0E0D0E064917F018FEFE81AF80A58
:10551000662361F0D801ED91FC910190F081E02DBE
:10552000C8010995C80FD91FF701EDCFCE01CDB73E
:10553000DEB7E6E00C94282F0E94622A0895DC0171
:10554000ED91FC910190F081E02D099508950F9364
:105550001F93CF93DF93EC016DE00E949F2A8C0193
:105560006AE0CE010E949F2A800F911FDF91CF91A8
:105570001F910F9108950F931F93CF93DF93EC0129
:105580000E94792A8C01CE010E94A72A800F911FC8
:10559000DF91CF911F910F9108950F931F93CF9398
:1055A000DF93EC010E94622A8C01CE010E94A72A9F
:1055B000800F911FDF91CF911F910F9108950F934D
:1055C0001F93CF93DF93EC010E949F2A8C01CE01A1
:1055D0000E94A72A800F911FDF91CF911F910F91F9
:1055E0000895A1E2B0E0E7EFFAE20C94062F7C0107
:1055F000C42EE52FCB01D22E19A221E02D1510F0DB
:105600002AE0D22E8E010F5D1F4F8D2C912CA12CE4
:10561000B12C6C2D7E2FA50194010E94BF2E8C2DE4
:10562000D29E80191124015011098A3010F4805D36
:1056300001C0895CF80180832115310541055105C0
:1056400021F0C22EE32FCA01E4CFB801C7010E94A6
:10565000622AA196ECE00C94222FA0E0B0E0E3E3F4
:10566000FBE20C940A2FEC016A017B012115310544
:1056700041F4E881F9810190F081E02D642F0995D2
:105680001DC02A303105A9F477FF12C06DE20E94D7
:105690009F2A8C0144275527BA014C195D096E09D0
:1056A0007F092AE0CE010E94F12A800F911F06C0D7
:1056B0002AE0B701A601CE010E94F12ACDB7DEB7DC
:1056C000E8E00C94262F9A01AB01662757FD609500
:1056D000762F0E942D2B08950F931F93CF93DF9366
:1056E000EC019A01AB01662757FD6095762F0E9469
:1056F0002D2B8C01CE010E94A72A800F911FDF91D4
:10570000CF911F910F9108952115310549F4DC01C6
:10571000ED91FC910190F081E02D642F09950895A1
:105720000E94F12A08959A01462F50E060E070E04F
:105730000E94842B08959A01AB0160E070E00E9402
:10574000842B08950F931F93CF93DF93EC010E9456
:10575000842B8C01CE010E94A72A800F911FDF911C
:10576000CF911F910F9108950F931F93CF93DF93C4
:10577000EC019A01AB0160E070E00E94842B8C0187
:10578000CE010E94A72A800F911FDF91CF911F9118
:105790000F9108950F931F93CF93DF93EC019A011C
:1057A000462F50E060E070E00E94842B8C01CE0117
:1057B0000E94A72A800F911FDF91CF911F910F9117
:1057C0000895FC0124853585F901E05CFF4F808157
:1057D0009181F901EE5BFF4F20813181821B930B98
:1057E0008F7399270895FC0184859585FC01E05C01
:1057F000FF4F40815181FC01EE5BFF4F20813181E1
:105800004217530741F00190F081E02DE80FF91F96
:10581000808190E008958FEF9FEF0895FC018485CB
:105820009585FC01E05CFF4F40815181FC01EE5BFE
:10583000FF4F208131814217530779F0A081B18158
:10584000A80FB91F8C91208131812F5F3F4F2F739B
:1058500033273183208390E008958FEF9FEF0895E1
:10586000FC0181A1882329F0A489B5898C9186FF48
:10587000FBCF11A20895CF93DF93FC0126853785D6
:10588000D901A05CBF4F8D919C91119701968F73A8
:105890009927E901CE5BDF4F48815981841795072D
:1058A000D9F30D90BC91A02DA20FB31F6C93A685C8
:1058B000B785A05CBF4F11969C938E93A689B7893C
:1058C0002C9181E090E0078C02C0880F991F0A9408
:1058D000E2F7282B2C9381E081A30488F589E02D41
:1058E00080818064808381E090E0DF91CF91089592
:1058F00008951F920F920FB60F9211242F933F938A
:105900004F938F939F93EF93FF938091C00082FDFD
:105910001CC04091C60080918C0690918D06019626
:105920008F73992720918E0630918F0682179307E7
:1059300071F0E0918C06F0918D06E45BF94F4083A5
:1059400090938D0680938C0602C08091C600FF91D3
:10595000EF919F918F914F913F912F910F900FBE9B
:105960000F901F90189586EE95E00E94E12B892BF1
:1059700011F00E94782C08951F920F920FB60F928B
:1059800011242F933F938F939F93EF93FF93209135
:1059900048063091490680914A0690914B06281797
:1059A000390731F48091C1008F7D8093C10014C00C
:1059B000E0914A06F0914B06E85FF94F2081809113
:1059C0004A0690914B0601968F73992790934B0648
:1059D00080934A062093C600FF91EF919F918F918B
:1059E0003F912F910F900FBE0F901F901895A0E040
:1059F000B0E0EDEFFCE20C94062FFC011382128262
:105A000088EE93E0A0E0B0E084839583A683B7831B
:105A10008CEB93E0918380837587648757874687F3
:105A2000318B208B138B028BF58AE48AD78AC68A46
:105A3000B18EA08E938E828E8F85848F8889858F7C
:105A40008989868F8A89878F8B8980A3ECE00C9463
:105A5000222FCF92DF92EF92FF92CF93DF93EC0150
:105A60006A017B01411581EE580761057105F9F066
:105A7000EC89FD8981E090E008A002C0880F991FA1
:105A80000A94E2F7808360E079E08DE390E0A7017B
:105A900096010E94BF2E21503109410951095695A6
:105AA000479537952795211580E1380798F0EC89BF
:105AB000FD89108260E874E88EE190E0A70196010C
:105AC0000E94BF2E21503109410951095695479531
:105AD00037952795E889F9893083EA89FB892083FE
:105AE00019A2EE89FF89408181E090E09C010C8C35
:105AF00002C0220F331F0A94E2F7422B4083EE8943
:105B0000FF8940819C010D8C02C0220F331F0A9433
:105B1000E2F7422B4083EE89FF8940819C010E8C85
:105B200002C0220F331F0A94E2F7422B4083EE8912
:105B3000FF8920810F8C02C0880F991F0A94E2F719
:105B4000809582238083DF91CF91FF90EF90DF904B
:105B5000CF900895BF92CF92DF92EF92FF92CF93B2
:105B6000DF93EC016A017B01B22E411581EE5807EB
:105B700061057105F9F0EC89FD8981E090E008A0EC
:105B800002C0880F991F0A94E2F7808360E079E0F1
:105B90008DE390E0A70196010E94BF2E21503109AC
:105BA000410951095695479537952795211580E16B
:105BB000380798F0EC89FD89108260E874E88EE17E
:105BC00090E0A70196010E94BF2E215031094109A2
:105BD00051095695479537952795E889F989308376
:105BE000EA89FB892083E88DF98DB082EE89FF89EF
:105BF000408181E090E09C010C8C02C0220F331F99
:105C00000A94E2F7422B4083EE89FF8940819C0190
:105C10000D8C02C0220F331F0A94E2F7422B4083FF
:105C2000EE89FF8940819C010E8C02C0220F331F38
:105C30000A94E2F7422B4083EE89FF8920810F8C82
:105C400002C0880F991F0A94E2F78095822380830F
:105C5000DF91CF91FF90EF90DF90CF90BF900895AC
:105C60008F929F92AF92BF92CF92DF92EF92FF926C
:105C70000F931F9381E08F9385E08F9387E08F933D
:105C800083E08F9384E08F93E6EC8E2E912CF2ECE0
:105C9000AF2EB12CA1ECCA2ED12CB0ECEB2EF12CF6
:105CA00004EC10E025EC30E048E056E06CE476E0EF
:105CB00086EE95E00E94F72C0F900F900F900F90BA
:105CC0000F901F910F91FF90EF90DF90CF90BF90BA
:105CD000AF909F908F9008950E942A290E94802261
:105CE000C3EBDCE20E9423252097E1F30E94B32C52
:105CF000F9CFA29FB001B39FC001A39F700D811D7A
:105D00001124911DB29F700D811D1124911D0895C4
:105D10000E94792EA59F900DB49F900DA49F800D99
:105D2000911D11240895B7FF0C94882E0E94882E8F
:105D3000821B930B0895DB018F939F930E94882E03
:105D4000BF91AF91A29F800D911DA39F900DB29F17
:105D5000900D1124089597FB072E16F4009407D098
:105D600077FD09D00E943D2F07FC05D03EF49095A9
:105D700081959F4F0895709561957F4F0895A1E299
:105D80001A2EAA1BBB1BFD010DC0AA1FBB1FEE1FB5
:105D9000FF1FA217B307E407F50720F0A21BB30B00
:105DA000E40BF50B661F771F881F991F1A9469F77C
:105DB00060957095809590959B01AC01BD01CF01D8
:105DC0000895052E97FB1EF400940E94F82E57FDAF
:105DD00007D00E94BF2E07FC03D04EF40C94F82E7F
:105DE00050954095309521953F4F4F4F5F4F089507
:105DF00090958095709561957F4F8F4F9F4F089537
:105E00002F923F924F925F926F927F928F929F92CA
:105E1000AF92BF92CF92DF92EF92FF920F931F93B8
:105E2000CF93DF93CDB7DEB7CA1BDB0B0FB6F89469
:105E3000DEBF0FBECDBF09942A88398848885F84A9
:105E40006E847D848C849B84AA84B984C884DF801A
:105E5000EE80FD800C811B81AA81B981CE0FD11DFE
:105E60000FB6F894DEBF0FBECDBFED010895EE0F63
:105E7000FF1F0590F491E02D0994AA1BBB1B51E173
:105E800007C0AA1FBB1FA617B70710F0A61BB70BAA
:105E9000881F991F5A95A9F780959095BC01CD014F
:105EA00008958F929F92AF92BF92CF92DF92EF921E
:105EB000FF92CF93DF93EC01688179818A819B8186
:105EC000611571058105910521F464E279ED8BE599
:105ED00097E02DE133EF41E050E00E94E12E4901CF
:105EE0005A019B01AC01A7EAB1E40E94882E6B0124
:105EF0007C01ACEEB4EFA50194010E94962EC60E73
:105F0000D71EE81EF91EF7FE06C081E0C81AD108A8
:105F1000E10880E8F80AC882D982EA82FB82C701D8
:105F2000B6019F77DF91CF91FF90EF90DF90CF90F8
:105F3000BF90AF909F908F9008950E94512F089529
:105F400086E091E00E94512F0895609306017093BE
:105F50000701809308019093090108952F923F92C1
:105F60005F926F927F928F929F92AF92BF92CF92E9
:105F7000DF92EF92FF920F931F93CF93DF938B01EA
:105F8000EA016115710521F0DB018C9311969C9358
:105F9000209739F09E01225031092332310508F053
:105FA000D8C07C016701BFEFCB1ADB0A5601F701AD
:105FB0006080862D90E00E94E030892B11F0760100
:105FC000F1CFFDE26F120AC0570182E0A80EB11CAA
:105FD000D70111966C90772473940BC0BBE26B12BF
:105FE00007C05701E2E0AE0EB11CD70111966C90CC
:105FF000712CCE018F7E892B89F4B0E36B1237C0F0
:10600000F50180818F7D8835D1F46180F2E0AF0E9B
:10601000B11C872D8260782EC0E1D0E0CA30D10556
:1060200051F1C031D10521F0C830D10599F409C032
:10603000CC24CA94DC2CEC2CAFE0FA2E22C02097A2
:1060400069F7C8E0D0E0CC24CA94DC2CEC2CFFE14A
:10605000FF2E17C06FEF7FEFCB019E01442737FD66
:106060004095542F0E94BF2E69017A010AC02097E3
:10607000A9F6CAE0D0E0E9E9CE2EDC2CEC2CE9E16F
:10608000FE2EF50160E020E030E0A9014E01AA24D7
:1060900097FCA094BA2C1F0170ED572E560CA9E066
:1060A000A51570F48FEB860D8A3118F499EC592EF2
:1060B00006C08FE9860D8A3148F589EA582E560CBC
:1060C000852D90E08C179D070CF56F3FD9F0C21617
:1060D000D306E406F50698F0C501B4010E949B2E94
:1060E0009B01AC01852D90E0A0E0B0E0280F391FA6
:1060F0004A1F5B1F281739074A075B0710F46FEF29
:1061000001C061E03196D1016C90C5CF0115110538
:1061100051F0662311F0319703C071FE04C032972D
:10612000D801ED93FC9370FE07C0509540953095D3
:1061300021953F4F4F4F5F4F67FF10C082E290E0C5
:1061400090939106809390066FEF7FEF8FEF9FEF14
:1061500007C060E070E080E090E002C0B901CA01D1
:10616000DF91CF911F910F91FF90EF90DF90CF9033
:10617000BF90AF909F908F907F906F905F903F9077
:106180002F900895FC0188279927E89421912032C7
:10619000E9F3293010F02E30C8F32B3241F02D32C4
:1061A00039F4689404C00E941431820F911D21912A
:1061B00020532A30C0F31EF4909581959F4F089587
:1061C000911150C0803219F089508550D0F7089550
:1061D00048EC53E00E94ED300895FA01A191B0819E
:1061E000009719F41097E1F0CD01DC01CD010D907D
:1061F000002011F4C00113C0FB012191222319F0EA
:106200002015D9F7F3CFFB012191201519F41E9227
:10621000119606C02223C1F70D900020A1F7D001EE
:10622000FA01A193B08308957AE0979F902D879FFC
:10623000802D910D11240895F999FECF92BD81BD55
:10624000F89A992780B50895262FF999FECF1FBA9D
:1062500092BD81BD20BD0FB6F894FA9AF99A0FBE8F
:0E62600001960895992788270895F894FFCF96
:10626E0000009206200001000000FF000200020064
:10627E000200020002000200020002000200020000
:10628E00020002000200020002000280250000054A
:10629E00400AA1204EA50020244EA52C2330C0126A
:1062AE0000001A400AA1204EA5001B1E27522C23C7
:1062BE00308025000005400AA1204EA50020244E66
:1062CE00A52C2330004B000006400AD0009D49004B
:1062DE007B289D492C233000E1000005400A450132
:1062EE00D7DC03B81E0EBF00232E48E801008A40FB
:1062FE000A6001555502AD1E20000023C8015458F6
:10630E002074696D656F75742100596573004E6F49
:10631E00002C00386368004E2F41002C205B005D7E
:10632E002028002900486F70206368616E6E656CCE
:10633E00200020402000456E746572696E672061F2
:10634E0064617074697665206368616E6E656C2039
:10635E0073656C656374696F6E2C207069636B690D
:10636E006E673A007363616E6E6572206D6F646561
:10637E00004E4F5420454E41424C45440053656EED
:10638E0064696E672073657474696E677320746FC9
:10639E002052580A00526573657474696E672073D3
:1063AE00657474696E6773206F6E2052580A0041CF
:1063BE00626F727465642065646974730A00696E35
:1063CE0076616C69642073656C656374696F6E00C9
:1063DE000D0A496E76616C696420696E7075742061
:1063EE002D206469736361726465642107005365CF
:1063FE007474696E677320736176656420746F20A0
:10640E00454550524F4D0A0052657665727465646B
:10641E002073657474696E67732066726F6D2045A4
:10642E004550524F4D0A004C6F61646564206661A1
:10643E0063746F72792064656661756C74730A009B
:10644E004B657920616E64206368616E6E656C7356
:10645E002072616E646F6D697A65640A004F7065B3
:10646E006E4C52536E672054582073746172746967
:10647E006E672000206F6E20485720006D6F647588
:10648E006C65206C6F636B65643F00342B34003891
:10649E0000382B340031320031322B3400313600CB
:1064AE0050504D0052535349005344410053434CF6
:1064BE0000525844005458440041494E004C424545
:1064CE0045500053504B54524D00534255530053B8
:1064DE00554D44004C4C494E440000070B0C101116
:1064EE001500B7012B032F033103350338033D038A
:1064FE00B7014003440349034D03510355035903A8
:10650E005D0363036A036F0374038D028D028D02B4
:10651E008D02160A13223129000000003B2C402A5E
:08652E00E12B0E2CF32B302CA5
:107E00000F92CDB7DEB7112484B714BE81FFF1D035
:107E100082E08093C00088E18093C10086E0809377
:107E2000C20080E18093C4008EE0CDD088249924E4
:107E3000CC24C394F5E0DF2EE1E1EE2E73E0F72EC3
:107E4000B6D0082F813479F4B2D08983C2D0898129
:107E5000823811F481E005C0813811F485E001C059
:107E600083E09ED09AC0823411F484E103C085344B
:107E700019F485E0B6D091C0853561F498D0082F0B
:107E800010E095D090E0982E8824802A912A880CC2
:107E9000991C82C0863521F484E0A3D080E0E1CF34
:107EA000843609F04CC083D082D0A82E80D0B82E62
:107EB00000E011E07CD0F80181938F01AE16D1F77C
:107EC00088D0FB2DF53489F4E0E0F1E00BC0F9999E
:107ED000FECF92BC81BC0894811C911C819180BD15
:107EE000FA9AF99AEA1598F358C08B2D863409F05E
:107EF00054C0F401F7BEE89507B600FCFDCFF401CD
:107F0000A0E0B1E02C9130E011968C91119790E0B7
:107F1000982F8827822B932B12960C01C7BEE895C9
:107F20001124329681E0A038B80761F7F401D7BE7A
:107F3000E89507B600FCFDCFE7BEE8952EC0843774
:107F4000F1F435D034D0182F32D0B82E42D0FB2DDA
:107F5000F63421F4F40105914F010CC0FB2DF534EA
:107F600049F4F999FECF92BC81BC0894811C911C04
:107F7000F89A00B5802F14D0115049F70EC08537FC
:107F800039F427D08EE10CD085E90AD08FE069CF93
:107F9000813511F488E017D01CD080E101D050CF9A
:107FA0009091C00095FFFCCF8093C600089580910A
:107FB000C00087FFFCCF8091C00084FD01C0A89560
:107FC0008091C6000895E0E6F0E098E19083808318
:107FD0000895EDDF803219F088E0F5DFFFCF84E10E
:107FE000DFCF1F93182FE3DF1150E9F7F2DF1F9166
:0E7FF0000895282E80E0E7DFEE27FF27099492
:027FFE0001057B
:0400000300007E007B
:00000001FF
